:020000040800F2
:1000000000800120210300088747000849470008B5
:1000100085470008452C0008EF610008000000003B
:1000200000000000000000000000000097470008EA
:100030008D2C000800000000954700085D4900086D
:100040003B0300083B0300083B0300083B03000898
:100050003B0300083B0300083B0300083B03000888
:100060003B0300083B0300083B0300083B03000878
:100070003B0300083B0300083B0300083B03000868
:100080003B0300083B0300083B030008000000009E
:100090000000000000000000000000003B0300081A
:1000A0003B0300083B0300083B0300083B03000838
:1000B0003B0300083B0300083B0300083B03000828
:1000C0003B0300083B0300083B0300083B03000818
:1000D0003B0300083B0300083B030008000000004E
:1000E0003B0300083B0300083B030008000000003E
:1000F0000000000000000000000000003B030008BA
:10010000000000003B0300083B0300083B0300081D
:1001100000000000000000000000000000000000DF
:100120003B0300083B0300083B0300083B030008B7
:100130003B03000800000000000000000000000079
:1001400000000000000000000000000089470008D7
:100150003B0300083B0300083B0300083B03000887
:100160003B0300083B030008000000000000000003
:10017000000000000000000000000000000000007F
:10018000000000003B030008000000000000000029
:100190003B03000800F002F800F0B8F80AA090E86D
:1001A000000C82448344AAF10107DA4501D100F032
:1001B000ADF8AFF2090EBAE80F0013F0010F18BF47
:1001C000FB1A43F00103184760C3000080C300001E
:1001D0000A444FF0000C10F8013B13F0070408BF6D
:1001E00010F8014B1D1108BF10F8015B641E05D00B
:1001F00010F8016B641E01F8016BF9D113F0080FC0
:100200001EBF10F8014BAD1C0C1B09D16D1E58BF51
:1002100001F801CBFAD505E014F8016B01F8016B88
:100220006D1EF9D59142D6D37047000000230024FB
:1002300000250026103A28BF78C1FBD8520728BFF6
:1002400030C148BF0B6070476E2900F07686702978
:1002500000F0858166290AF01F8765290AF01C874E
:1002600067290AF0198761290AF0188703681B0AB1
:1002700028BF41F08001692900F0F680642900F070
:10028000F380752900F0F0806F2900F04787782906
:1002900000F05181E92900F0E186E42900F0DE86D2
:1002A000F52900F0DB86EF2900F04487F82900F0FB
:1002B00050810368DB0928BF41F08001632901F008
:1002C0006185732901F06685E32901F07185F329C1
:1002D00001F07685002070471FB50AF0D8FE9DE832
:1002E000030000F039FD01F0CBFF040000200021E5
:1002F0000AF07CFE401C6060002000210AF060FED5
:10030000E06001F07DF800F0F5FC1FBD09F088FB0E
:100310001146FFF7E1FF02F088FC09F087FD0000BD
:100320000648804706480047FEE7FEE7FEE7FEE78F
:10033000FEE7FEE7FEE7FEE7FEE7FEE7F14900081D
:100340009501000870B5064600F0E6FC056806F168
:100350000B0020F00704B4429CBF002070BD2B4668
:100360006A68BAB11068A04210D304F1080188424B
:100370003CBF5068586007D351681019416011683C
:10038000091B016058601460101D70BD134652684F
:10039000002AE7D12146284600F0CAFC0028DED119
:1003A00070BD70B50446051F00F0B6FC0068002C57
:1003B00014BF446870BD002C18BFAC423CBF20463F
:1003C0006468F8D301680A18AA4218BF456003D1CF
:1003D0002A6805461144016028684119A1421CBFE2
:1003E0006C6070BD6168696021680844286070BDF8
:1003F000B2F120030AD5C2F1200301FA02F120FA7A
:1004000003F300FA02F041EA0301704700FA03F136
:100410004FF00000704700001CB50C46064B7B44B3
:1004200069460090204600F0A2FD0446002069467F
:1004300000F0B0FD20461CBD730B00000FB41CB5CE
:10044000084B06AA7B4469460090059800F08FFD92
:1004500004460020694600F09DFD20461CBC5DF866
:1004600014FB00004D0B00002DE9F041064600246E
:1004700010687529314616A510D000F0CAFC002876
:1004800002DA404213A507E031688A0701D512A5B8
:1004900002E0490704D511A5012401E000F0C2FCE7
:1004A00000210A2206F1240709E0B0FBF2FCB0FBB0
:1004B000F2F302FB1C00303078541846491C002827
:1004C000F3D123462A463046BDE8F04100F0DCBCBB
:1004D000000000002D0000002B00000020000000A4
:1004E000F0B40D460188090502D5214C7C4402E098
:1004F0001F4C7C440E34002100F1240608E002F079
:100500000F071209E75D42EA03721B097754491C81
:1005100052EA0307F3D102780023120704D5702DA5
:1005200006D009B1022311342246F0BC00F0ACBC65
:1005300001231034F8E770B504460D4621461068D3
:1005400000F070FC024629462046BDE870400023BA
:10055000C6E7D21D22F00703D3E90023C0E70368F2
:10056000126843F0200303600823C3610023B7E748
:1005700064BD00002DE9F05F894604464FF0000A93
:10058000DFF874B1FB44C0F820A02046E16888473A
:10059000002874D0252806D0D4E901219047206A8C
:1005A000401C2062F1E700265F462046E16888474C
:1005B0002028054607DB312D05D2781910F8200CCC
:1005C00008B10643F1E7B00701D526F00406C4F8E8
:1005D0001CA00027C4F818A02A2D09D0284609F02D
:1005E00027FA38B304EB8708303DC8F8185019E0F3
:1005F00059F8041B204604EB87029161E1688847A3
:10060000012F054618D1E069002820DA26F02006DF
:100610001DE0D8F8180000EB800005EB40003038F2
:10062000C8F818002046E1688847054609F000FA36
:100630000028EED1012F0AD02E2D08D12046E168E6
:1006400088477F1C0546022F46F02006C4DBA069C0
:10065000002803DA404246F00106A061F00701D00D
:1006600026F010066C2D0BD0682D09D04C2D39D0FA
:100670006A2D35D0742D35D07A2D33D016E038E080
:10068000E1682F4620468847B842054609D16C2FBD
:1006900026D04FF48060E16806432046884705462F
:1006A00004E06C2F1AD04FF4807006430DB3A5F10F
:1006B0004100192802D8203546F400664A462946EA
:1006C000204626604E46FFF7BFFD80B101280BD0C3
:1006D000F61D26F0070000F1080956E74020E4E780
:1006E0008020D8E70020D6E706F104094DE7284628
:1006F00052E7206ABDE8F09FF4BC00000FB400B5DB
:100700008DB010A9099000910B904FF0FF300A9026
:1007100000200C90064878440690064878446A46C3
:1007200007900F9909A800F023FD0DB05DF814FBA8
:10073000770A00008F0A00002DE9FF5F1D464FF089
:10074000FF3B91464FF000085F46D5E90146A96995
:1007500001987F1C8847296A824688470028F6D17D
:10076000BAF1FF3F0CD0002E24F4C06419DD6006FE
:1007700014D5BAF12B0F09D0BAF12D0F0ED103E029
:10078000584604B0BDE8F09F44F48064A96901981C
:100790007F1C8847761E8246002E02DDBAF1300F9C
:1007A00003D0B9F1000F26D032E0A969761E019876
:1007B0007F1C44F400748847002E824605DDBAF1A0
:1007C000780F06D0BAF1580F03D0B9F1000F10D04E
:1007D0001EE0B9F1000F02D0B9F1100F18D1A969CC
:1007E000761E01987F1C24F40074884782461020EE
:1007F00002E0082000E00A20814609E0A96908FB20
:100800000908761E01987F1C44F4007488478246CC
:10081000002E05DD4946504600F096FC0028EDDA32
:10082000E96901988847A00502D46FF00100A8E7A4
:10083000E00725D1600613D5600502D5C8F1000098
:1008400000E0404629680A1D2A600968220501D592
:10085000087015E0220701D5088011E008600FE05C
:100860002868011D29600068210502D580F80080F4
:1008700006E0210702D5A0F8008001E0C0F8008062
:1008800038467EE770B50446C068810713D08006FD
:1008900001D5A56A04E0A169606808442169451A88
:1008A000204600F069FD002206462946204600F059
:1008B0008FFC304670BD002070BD70B510B1BDE832
:1008C0007040DFE70025074C6E1E07E02046FFF76B
:1008D000D9FF00B13546206D20F00104002CF5D180
:1008E000284670BD4C7000202DE9F0410C460746AB
:1008F0001646104600F078F82078611C61280AD06E
:10090000722802D077283CD102E00125002405E0BE
:100910000225042402E0082448F2020511F8010B24
:100920002B2806D0622809D011F8010C74280AD0AF
:100930000BE045F0030544F00204EFE745F0040541
:1009400044F00104EAE744F010043846214609F077
:10095000B5F8411C15D00021316171604FF4007170
:10096000F560F1617061200704D530460222002154
:1009700000F02EFC306D40F0010030653046BDE8DF
:10098000F0810020FBE72DE9F0410D460646104CB2
:10099000206DC10704D0410804D020F00104F7E71E
:1009A00022460EE05420FFF7CDFC07000ED0206D4C
:1009B00047F00101084354212065384600F032F920
:1009C0003A4629463046BDE8F0418DE70020D6E79B
:1009D0004C70002011B14FF4807201E04FF480623E
:1009E0004FF4007300F070BC2DE9F04704464FF05F
:1009F00000094FF0FF37C568D4E90486A80707D07F
:100A0000204600F0B9FC304609F01AF8002802DA56
:100A10003846BDE8F087280502D54046FFF7C1FCFF
:100A20004C21204600F0FEF8206D20F001002065EA
:100A30004846EEE72DE9F041074615460E461020E0
:100A4000FFF780FC04000AD06760C4E9026500F08B
:100A500067F90168216004600020BDE8F081012091
:100A6000FBE710B5431C02E010F8011B71B18107D0
:100A7000FAD14FF0013202C88C1A8C4314EAC21129
:100A8000F9D0C01A0A0603D0C01E10BDC01A10BD8E
:100A90000A0401D0801E10BD0902FCD0401E10BD0A
:100AA00040EA010370B59B072ED14FF00136042AAE
:100AB0002AD308C810C99D1B9D43121F15EAC615ED
:100AC00017D0D8B2E1B2401A50EA056110D198B2FD
:100AD000A1B2401A50EA05410AD123F07F4024F028
:100AE0007F41401A50EA052102D1180EA0EB146094
:100AF00070BDA342DBD018BA21BA884201D90120C7
:100B000070BD4FF0FF3070BD0AB9002070BD10F805
:100B1000013B11F8014B63B1A3420AD1521E08D028
:100B200010F8013B11F8014B1BB1A34201D1521E39
:100B3000EDD1181B70BD032A40F2308010F0030C79
:100B400000F0158011F8013BBCF1020F624498BF20
:100B500011F801CB00F8013B38BF11F8013BA2F1BD
:100B6000040298BF00F801CB38BF00F8013B11F038
:100B7000030300F02580083AC0F0088051F8043BD8
:100B8000083A51F804CBA0E80810F5E7121D5CBF45
:100B900051F8043B40F8043BAFF30080D20724BF78
:100BA00011F8013B11F801CB48BF11F8012B24BF0C
:100BB00000F8013B00F801CB48BF00F8012B70475B
:100BC00010B5203AC0F00B80B1E81850203AA0E8E8
:100BD0001850B1E81850A0E81850BFF4F5AF5FEA1C
:100BE000027C24BFB1E81850A0E8185044BF18C9CF
:100BF00018C0BDE810405FEA827C24BF51F8043B76
:100C000040F8043B08BF7047D20728BF31F8023BC9
:100C100048BF11F8012B28BF20F8023B48BF00F85D
:100C2000012B70474FF0000200B5134694469646DC
:100C3000203922BFA0E80C50A0E80C50B1F12001EF
:100C4000BFF4F7AF090728BFA0E80C5048BF0CC09D
:100C50005DF804EB890028BF40F8042B08BF7047FB
:100C600048BF20F8022B11F0804F18BF00F8012B6D
:100C7000704700004FF0013C50F8042B51F8043B42
:100C80009A4221D1A2EB0C03934313EACC1317D160
:100C900050F8042B51F8043B9A4215D1A2EB0C03F7
:100CA000934313EACC130BD150F8042B51F8043BB7
:100CB0009A4209D1A2EB0C03934313EACC13DBD085
:100CC0004FF00000704700BFD01A01BAB1FA81F1AD
:100CD00001F0180122FA01F0CB40C1F12001DBB292
:100CE000C0B2C01A2CFA01F3D11A914311EAC31110
:100CF000E6D1704770B5064C7C44064D7D4403E058
:100D0000206820448047241DAC42F9D170BD00000A
:100D100078B900007CB90000004870474871002095
:100D2000004870474C71002070477047704770470B
:100D300038B504460A460020694601F076FA0028D4
:100D400008BF38BD02460099204600F01DFC012076
:100D500038BD012001F03FBAF8B501F05BFA054655
:100D600000200C46102000BF0646A819A0420DD94D
:100D700032466946002001F058FA070008BF01F02A
:100D80002AFA0098A04218BF0546C419FFF7C4FF0D
:100D900005600746F01D20F007004619284600F0C0
:100DA0000AF8B44208BFF8BDA21B31463868BDE856
:100DB000F84000F0E9BB00210160C0E90110704774
:100DC0001020704770B5044685690068C10601D5DA
:100DD000302600E02026C00707D070BDD4E90121ED
:100DE00030469047206A401C20626D1EF6D570BDCB
:100DF00070B5044685690078C00707D170BDD4E995
:100E0000012120209047206A401C20626D1EF6D5EB
:100E100070BD09684A0501D540B27047C905FCD5C7
:100E200000B2704709684A0501D5C0B27047C905CC
:100E3000FCD580B2704770B50C460546012A05D036
:100E40002878800600D5EA69002302E0012305E046
:100E50005B1C934202D2E05C0028F9D1A869E61835
:100E6000C01AA861286A184428622846FFF7AAFF1A
:100E700004E0D5E9012114F8010B9047B442F8D3FE
:100E80002846FFF7B5FF70BD2DE9F0470D4699469E
:100E90009246044600F124080168880604D5E069FA
:100EA00021F01001216000E00120A84201DD471B74
:100EB00000E00027A1697A1902EB0900081AA06175
:100EC0002078C00602D42046FFF77CFF002608E009
:100ED000D4E901211AF806009047206A401C761CCC
:100EE00020624E45F4DB2078C0060AD52046FFF785
:100EF00069FF06E0D4E9012130209047206A401CB8
:100F00002062381EA7F10107F4DC07E0D4E90121D3
:100F100018F805009047206A401C2062281EA5F1A1
:100F20000105F3DC2046FFF763FF2078000602D5B9
:100F30000220BDE8F0870120FBE711680268006A23
:100F4000530501D508700AE0D30501D5088006E0F5
:100F5000130603D5C217C1E9000200E008600120B2
:100F60007047000001694A1C02610878704700B5AB
:100F70008FB0CDE901310021059105497944CDE9D2
:100F8000031011466846FFF7F5FA0FB000BD0000E8
:100F9000E5FFFFFF0A6802F8010B0A6070470000D6
:100FA0002DE9FF5F15468A460446DFF8AC80F84419
:100FB0000027D8E900103E46CDE9001010E03AF8CD
:100FC00016106A4602A801F0DAF8411C07D0217811
:100FD000890603D5E269391891420DD80744761C79
:100FE0002078800602D5E069B84205DDAE42E6DB36
:100FF0003AF816000028E2D1A069C01BA061204683
:10100000FFF7E0FED8E90010CDE90010002017E05E
:101010003AF818106A4602A801F0B1F8B0F1FF3FA3
:1010200081460BD000250DF1080B05E0D4E9012124
:101030001BF8050090476D1C4D45F7D308F10100E2
:10104000B0428046E4DB206A384420622046FFF745
:10105000CFFEBDE8FF9F0000DEB200002DE9F041A9
:101060008046D21D22F007020025D2E90002F529B0
:1010700015A614D0011E72F1000106DA0023D0EB90
:10108000030063EB020211A608E0D8F800108B07FA
:1010900001D50FA602E0490701D50EA6012511468C
:1010A000002408F1240704E000F088FA30323A55B1
:1010B000641C50EA0102F7D12B46324621464046D5
:1010C000BDE8F041FFF7E0BE000000002D00000089
:1010D0002B0000002000000030B4002100F12404A7
:1010E00008E002F00705D208303542EA4372DB0817
:1010F0006554491C52EA0305F3D10468002310A289
:10110000250708D504F020040C4304D0C46901234A
:101110000CA2641EC46130BCFFF7B6BE10B5044615
:1011200021461068FFF77EFE02462046BDE81040CB
:101130000023D1E7D21D22F00701D1E90023CBE73C
:1011400000000000300000003A2800D2303820F0C3
:101150002002412A01D3A2F13700884201D34FF087
:10116000FF307047026811441378016018467047D9
:10117000D1600549794451610449794411620021E3
:101180001161114600F020BEEDFFFFFFC904000011
:10119000426842B1016811F8013B23B1521EC0E917
:1011A0000012184670470121C160881E70474268CE
:1011B0005AB1C368016843B983688B4205D0491EA0
:1011C000521CC0E90012002070474FF0FF307047FA
:1011D0002DE9F041044616460D464769007B80071D
:1011E0002ED0384608F056FC50BB3EB3012E02D03C
:1011F000022E25D104E0204600F0A0FF05441DE0AA
:10120000384608F033FCE168002841F01001E16045
:1012100005DA204600F07CF80120BDE8F081C90322
:101220000BD56268E16A914200D81146A269114467
:101230002269891A814200DD08460544002D01DA41
:101240000220EAE7E16A6068E268814206D291031F
:10125000E06203D522F4003141F01002A6690027B4
:10126000AE4213DCE16A814201D90B4600E003463D
:1012700003EB060C2369ACEB030CAC4506DD8142A5
:1012800001D98C4600E084469C4505D1A7602760C3
:1012900042F02000A5620DE0AD1BE669AE1B814265
:1012A000A66000D90846C01A281A20605819606044
:1012B00022F0200003490840E060002084F84870D4
:1012C000ABE70000BFCFD7FF70B5C468A50713D048
:1012D000650211D4B2F5807F09D0B2F5007F06D047
:1012E000B2F5806F08D1012300F1240106E05D1EF4
:1012F0006FF07F46B54201D3012070BD0161C3612B
:10130000416024F470611143C160002070BD000091
:10131000C16821F4001141F08001C16000218160A9
:10132000016070472DE9F047814614460E464FF0A4
:10133000FF383248D5685769054209D03846A16957
:1013400008F098FC002811DB2C48C0430540E560FC
:101350002B4632464946384608F0A0FCA16920F0E9
:101360000042B21A11440028A16103D02046FFF7C1
:10137000CFFF4046BDE8F08770B504460569C06AF6
:101380006168884200D80846E16821F42011E160D4
:10139000C90312D5A84208D02246411B2846FFF7B0
:1013A000C1FF10B14FF0FF3070BD0020E562C4E90D
:1013B0000150E06820F48030E060002070BD10B57E
:1013C0000446C06820F02000E060A16AA06988425D
:1013D0000DD02046FFF7D0FFE06820F4405040F0E9
:1013E0001000E060A06AA0612069E062606044F2E1
:1013F0004001E0688843E06010BD0000100002007A
:1014000010B542485421FFF70DFC41485421FFF725
:1014100009FC40485421FFF705FC3F493B483C4A42
:101420003F4B08603D490A603A491960531C036507
:10143000481C1065012008653B48344A39A17844AE
:10144000FFF752FA20B9384878440A3800F0BCFE59
:1014500037482F4A35A17844FFF746FA20B9344877
:1014600078440A3800F0B0FE32482A4A2FA1784466
:10147000FFF73AFA20B92F4878440A3800F0A4FE62
:1014800040232248DC0000212246FFF71DFF20B147
:1014900025487844543800F097FE1D4822464023E2
:1014A0000021FFF711FF20B121487844543800F0A3
:1014B0008BFE1848224610230021FFF705FF002865
:1014C00006D01C487844BDE81040563800F07CBE79
:1014D00010BD104870B5006D20F001040B48FFF7F7
:1014E00083FA0B48FFF780FA0A48FFF77DFA09E014
:1014F000206D20F001052046FFF776FA2046FEF722
:1015000050FF2C46002CF3D170BD00004C70002021
:10151000A0700020F47000201004002014040020AB
:101520001804002072000000829E00007700000076
:10153000719E0000619E00002DE9F0410646FFF714
:10154000EFFB8046454613E016B1E068B0420ED18D
:1015500020682860D4E90101D8F800708847204647
:10156000FEF71FFFD8F80000B842EBD100E0254697
:101570002C68002CE8D1BDE8F08110B500F032FEF7
:10158000BDE8104000F01BBE034640688C460028B2
:1015900018BF88423CBF03464068F8D31868184417
:1015A000884207D00CF1030020F00700001D411A0B
:1015B000521A0146081D0A60FEF7F3BE30B5B0F1BD
:1015C0000A024FEA900E71F100034EEA817EB0EB01
:1015D0000E0061EB91014FEA101E4EEA017E10EB06
:1015E0000E0041EB11114FEA102E4EEA016E10EB86
:1015F0000E0041EB11214FEA104E4EEA014E10EB66
:101600000E0041EB1141401841F100014FEAD000BA
:1016100040EA41704FEAD10110EB80054FEA8104A6
:1016200044EA907444EB01046D1944EB0404521B2A
:10163000A3414FF0000348BF0A3200D530BD401C23
:1016400041F1000130BD10B5044600F011FE006804
:10165000005D00F0010010BD70472DE9FF4F0C4602
:101660001E464FF0FF378BB0D2E90001DDF86080F5
:101670000A908A46C1F30A5505B93D46002108463D
:101680004FF00000BAF1000F00F4400005DA00EB63
:1016900080004FF4400101EA50004FEA9059B9F13F
:1016A000010F00DDB9460A9850EA4A000ED044F610
:1016B0001050A5F2FF3545432F14B8F1000F1ED08E
:1016C0007542291E1EDDC9F100021CE0B8F1010FB0
:1016D0004FF0000001D0302103E0F24305E0215437
:1016E000401CB042FBDB30460022002121540B9904
:1016F000C1F80880C1E900200FB0BDE8F08FBD1B24
:101700006D1CDEE74A4600DA694206A800F000FEDA
:1017100006AB93E8070003AB83E8070050460A993D
:1017200000F0C8FE8DE80700A0F500501F380090BB
:101730000398002D09DD42F21F014A46084403A91F
:101740000390684601F027F908E0A0F500504A46EA
:101750001F3803A90390684601F031F98DE80700AE
:101760000004000C03D04FF0FF30410800E01046A9
:10177000B8F1000F03D00022009215461EE0751E3E
:1017800005D4FFF71BFF303262556D1EF9D5B34605
:101790000122084302D000227F1C04E02078302878
:1017A00001D100227F1E002A099786D01DE0112D4D
:1017B00007DAFFF703FF303262556D1C50EA010271
:1017C000F5D1084302D00098C8B10EE00021681E90
:1017D00005E0235C625C63542254401E491C814234
:1017E000F7DBAB46A81B401E0990002004F80B0055
:1017F0000B98099AC0F80880C0E9002B7CE71126F5
:101800004FF0000859E72DE9F04F88460446D21DF5
:1018100022F0070191B0D1E90001CDE90A0108F0F9
:1018200067F802460B98C00F01D02D2007E0206812
:10183000810701D52B2002E0202101EAC000032A04
:10184000099001D0072A05DB03464146204600F0F7
:101850001FFD0BE12078800601D5E06900E006203D
:10186000B8F1650F814606D0B8F1660F18D0B8F10F
:10187000670F70D131E00020B9F1110F009001DB4A
:10188000112301E009F101030AAA01A90CA8FFF73D
:10189000E4FEDDE90C70002609F10105834647E00E
:1018A00001204B4600904FF000470AAA01A90CA85E
:1018B000FFF7D3FEDDE90DB00C995D46002610B9A7
:1018C00009F101000D18B9EB050003D4C0F1FF3692
:1018D00009F10105A5EB09002BE0B9F1010F01DACF
:1018E0004FF001090020B9F1110F0090484601DDC9
:1018F000112300E003460AAA01A90CA8FFF7ADFED8
:10190000DDE90C704D4600268346207800070AD496
:10191000AB4500DA5D4601A8012D04DD411911F83F
:10192000011C302907D04F4502DA17F1040F04DA01
:10193000012082460FE06D1EEEE7002F02DCED1B5A
:101940003E4403E0781CA84200DD7D1CB81B00F17A
:10195000010A4FF000472078000703D4AA4501DBB5
:101960004FF0FF3A0021B7F1004F0DF143088DF819
:10197000431024D002202B23002F01DA7F422D2395
:101980000A21021EA0F1010000DC5FB197FBF1FC0F
:1019900097FBF1F201FB1C7C17460CF1300C08F8A8
:1019A00001CDEEE7A8F1010003702188090501D5FA
:1019B000452100E06521A0F1010800F8011C09980B
:1019C0000FA9A1EB0807FF1D00B10120411901EB90
:1019D000EA70A1693844081A401EA0612078C00648
:1019E00002D42046FFF7EEF9099828B1D4E9012185
:1019F0009047206A401C20622078C00622D52046ED
:101A0000FFF7E0F91EE0002E04DBB34502DD01A87C
:101A1000805D00E03020D4E901219047206A401C1D
:101A20002062761CAAF101005FEA000A0AD100F0E8
:101A300027FCC0680168405CD4E901219047206A16
:101A4000401C2062281EA5F10105DCDC07E0D4E97A
:101A5000012118F8010B9047206A401C2062381EB3
:101A6000A7F10107F3DC2046FFF7C2F9032011B00C
:101A700043E600002DE9F04F04460D46D21D22F04A
:101A8000070089B0D0E900974846394607F030FF93
:101A90000246F80F01D02D2307E02068810701D509
:101AA0002B2302E0202101EAC0038DF820300BB186
:101AB000012000E00020032A824601D0072A04DB2F
:101AC0002946204600F0E4FB3FE12078800601D45F
:101AD0000D2500E0E569C7F30A560D2D49DA00210E
:101AE0004FEA175B08464FF00000002F00F440005B
:101AF00007DA00EB80004FF4400100EBD07001EA00
:101B000060008115012901DD4FF0FF3100224FEA0D
:101B1000850CBCF1180F06D31346ACF118004FF03A
:101B20008052C24003E04FF4801323FA0CF30CF10F
:101B30000C0CBCF1200F04D3ACF1200C09FA0CF012
:101B400001E007FA0CF000294FF0004801DD18B958
:101B50000FE00ED140450CD319EB02095F4121B9CA
:101B6000404502D19F4329EA0209BBEB175F00D031
:101B7000761C2088000502D57B48784402E07A482C
:101B80007844193808AA302302F80A30037C0AF195
:101B90000101002E0AF1020A53546A4602DC4FF09A
:101BA000300101E04FF031014FF001088DF80010D5
:101BB00002D0A6F2FF3603E059EA470100D06B4E8F
:101BC000002D02DC2178090704D54FF002082E21F0
:101BD0008DF80110C44600210BE0C7F303433F0119
:101BE000C35C491C6D1E02F80830052908F1010884
:101BF00001DA002DF1DC00210CE000EB1973491C27
:101C00001B786D1E082902F808304FEA091908F1FF
:101C1000010801DA002DF0DC21688B0602D516E000
:101C2000A8F10108E04505DD02EB080313F8013CCB
:101C3000302BF5D0B8F1000F09DD02EB080313F8E3
:101C4000013C2E2B03D1090701D4A8F10108002D76
:101C500005DD3E2102F808106D1E08F10108407CE8
:101C6000002E02F8080008F1010804DA2D2076425F
:101C700002F8080002E02B2002F808000A214FF4C5
:101C80007A70864208F101080BDB96FBF0F33033E3
:101C900002F8083096FBF0F308F1010800FB136628
:101CA00001E0642E0CDB642096FBF0F3303302F885
:101CB000083096FBF0F308F1010800FB136601E021
:101CC0000A2E06DB96FBF1F0303002F8080008F12E
:101CD000010896FBF1F001FB1060303002F80800BB
:101CE000A16908F1010808EB050202EB0A00081AD5
:101CF000A0612078C00602D42046FFF763F8216A6D
:101D000008AE01EB0A00206204E0D4E9012116F8D4
:101D1000010B9047BAF1010AF7D22078C00602D52C
:101D20002046FFF74FF86E4609E016F8010B3E28F3
:101D30000FD0D4E901219047206A401C2062B8F1FD
:101D40000108F2D22046FFF753F809B00320BDE89E
:101D5000F08F206A2844206203E0D4E9012130207A
:101D600090476D1EEBD3F8E72DA7000002FCFFFFA4
:101D700010B5436913B1AFF3008001E0FFF75BF8E2
:101D8000012010BD127800F124010A7000224A706F
:101D90000122EDE711684FF0FF32E9E710B5436922
:101DA00013B1AFF3008001E0FFF7FAF8012010BD96
:101DB000128800F1240182840022C2840122EDE70E
:101DC00011684FF0FF32E9E72DE9F34F4FF0000AB9
:101DD0000C4656468DB001200C9001F10C000B9082
:101DE00062690B9801219047051E2DD0252D2CD01E
:101DF000216A8847C0B162690B9801219047216A26
:101E000088470028F7D16269411E0B98904700E08F
:101E1000761CA1690D988847216A88470028F7D168
:101E2000E1690D988847DBE7A1690D988847A842CA
:101E3000074601D1761CD3E7E1690D9888477F1CDE
:101E400002D1BAF1000F6FD06BE162690B980027E5
:101E50003D46394690472A2804D162690B980121F2
:101E600090470125DFF8D08262690B9801219047E5
:101E7000A0F130010A290AD24745E5DC07EB8701CA
:101E800000EB4107303FDFD445F01005ECE7E906F1
:101E900001D46FF000476C280AD04C2814D0682871
:101EA00015D06A280DD074281CD07A281AD01DE0CD
:101EB00062690B98012190476C2802D045F0040517
:101EC00014E045F002050DE045F020050AE06269E6
:101ED0000B9801219047682802D045F0080505E0DD
:101EE00045F4006562690B9801219047C4E90157E8
:101EF00065283DD019DC58287AD00CDC452837D02D
:101F000004DC252826D041289ED131E046282FD058
:101F1000472899D12CE05B2877D0612828D0632806
:101F20007CD0642823D15AE0F6E06F2848D008DC42
:101F300066281DD067281BD0692821D06E2816D1AD
:101F400027E0702845D0732868D0752847D07828B6
:101F50000DD14DE0A1690D988847252805463FF42D
:101F600069AFE1690D9888476D1C3FF46AAFD8E00E
:101F70000D9923466A466FF00100AFF30080C5E07B
:101F800045F0400023464FF000026060A80736D4B9
:101F90003EE0E8077FF447AF2068011D216000683C
:101FA000290501D506701BE7290701D5068017E72B
:101FB000A90703D5F117C0E9006111E706600FE733
:101FC00045F0400023464FF008026060A80716D491
:101FD0001EE040F60E0125EA0100606016E045F0C3
:101FE000400023464FF00A026060A80707D40FE0C4
:101FF00045F040006060A80708D5234610220D99DF
:102000006FF00100AFF3008080E007E0102223466C
:102010000D996FF00100FEF78FFB77E04FF000099C
:1020200063284F46C8464B46CB4602D05B2806D0B5
:1020300038E0E80601D40120A060012732E062699F
:10204000D4F80CB00B98012190475E2807D14FF0CF
:10205000010949466269D4F80CB00B989047216990
:1020600039B900210A4603AB43F82120491C08294D
:10207000FADBD8B3216949B308F1010862690B980A
:10208000012190475D28F4D1B9F1000F09D000205B
:1020900003A951F82020D24341F82020401C0828F1
:1020A000F7DB03AB2069002820794FEA40701ED08F
:1020B0005B462246CDF80080CDE901970D990028B6
:1020C0006FF0010020DAAFF300801FE0C11703AA10
:1020D00000EBD1614B1121F01F0102EB8302411A89
:1020E00013680120884003431360C7E719E00D9986
:1020F000224600286FF00100009702DAAFF300805B
:1021000004E0AFF3008001E0AFF3008000280ADABA
:10211000401C06D10C9820B14FF0FF300FB0BDE845
:10212000F08F5046FAE7E90701D10AF1010A0644A7
:1021300000200C9054E60000CCCCCC0C10B501462D
:10214000C268900703D0900607D5886A0AE000F0BD
:102150009BF801210160881E10BD8B6948681844F6
:102160000B69C01A91F848301BB191F84910401A18
:1021700010BD1103FCD50028FADD401E10BD70B55E
:1021800016460C46054600F073F8036893F8010103
:10219000012806D0FF2C0FD8185D68B101202C70E3
:1021A00070BDD3F807013246214603F207130344FA
:1021B0002846BDE8704018474FF0FF3070BD00283A
:1021C00001D000F04FB8704710B500F029F9BDE814
:1021D0001040FFF7F4BF10B500F03CF9BDE8104027
:1021E000FFF7EDBF10B5002102A000F0FFF80120BD
:1021F00010BD00005349475056464E3A2050757264
:1022000065207669727475616C20666E2063616CFE
:102210006C656400124B694600F580528A421A6070
:1022200001D8114670471960704730B50C4D6B46A8
:10223000A3F580532C6822449A420FD89B1A02F5CA
:10224000805003EBD37302EB6303984200D9184626
:10225000C01D20F007020C60101B2A6030BD00007A
:102260001C04002001491820ABBEFEE72600020036
:1022700010B500F005F8001D10BD00BF718D000005
:10228000004870475071002000487047647100207A
:102290002DE9F0411F46044603260168072A01F490
:1022A000006004DB08B116A505E016A503E008B13F
:1022B00015A500E015A521F010002060A069C01E42
:1022C000A0610FB1401EA0612046FEF77BFD4FB11B
:1022D000D4E9012138469047206A401C2062C01C86
:1022E000206206E0206AFAE7D4E9012115F8010B23
:1022F0009047761EF8D22046FEF77AFDBDE8F081C1
:102300004E414E006E616E00494E4600696E660099
:102310002DE9F047814616468AB0334878440DC807
:102320008DE80D0030487844801C03AC0DC884E86B
:102330000D0041F69B300844372190FBF1F290FBF1
:10234000F1F5A5F1800501FB12041B3C02D56442A6
:10235000012000E00020DFF890A080460027FA442A
:10236000AAF1BE0A0DE0E00709D03246684607EB45
:1023700047010AEB810100F022FB8DE807006410A1
:102380007F1C002CEFD1184F7F44AC3F18E0E807CA
:1023900014D007EB04100DF1180A90E80E008AE83B
:1023A0000E00C068F04201D198190890324606A983
:1023B00003A800F004FB03AB83E807006D10641C66
:1023C000002DE4D132466946B8F1000F03A802D0CF
:1023D00000F0E1FA01E000F0F2FAC9E90001C9F801
:1023E00008200AB0BDE8F0871CA0000070B50546C3
:1023F0000C460A2000E06D1C00F054F835B1287836
:102400000028F8D102E0641C00F04CF814B12078E8
:102410000028F8D1BDE870400A2000F043B8000061
:1024200010B5014602A0FFF7E1FF012010BD00003A
:1024300053494752545245443A2052656469726583
:1024400063743A2063616E2774206F70656E3A2062
:102450000000000010B5012805D0002103A0FFF7FF
:10246000C5FF012010BD09A1F8E7000053494752FC
:10247000544D454D3A204F7574206F662068656154
:1024800070206D656D6F7279000000003A2048651C
:102490006170206D656D6F727920636F72727570F7
:1024A0007465640008B569468DF800000320ABBE72
:1024B00008BD70475FEA400C08BF91F0000F4FEA7B
:1024C0008C234FEAC12243EA51514FEA1C5018BFF6
:1024D00000F5F0404FEA300018BF41F000415FEADC
:1024E0006C5C00F02980BCF1FF3F08BF40F08040E9
:1024F0007047130C06BF12044FF0100C4FF0000C85
:10250000130E04BF12020CF1080C130F04BF1201CA
:102510000CF1040C930F04BF92000CF1020CD30FCA
:1025200004BF52000CF1010C11464FF00002A0F163
:102530001F00A0EB0C00704711F0004F08BF704760
:1025400031F000413FF4D5AF0B0C06BF09044FF04A
:10255000100C4FF0000C0B0E04BF09020CF1080C1C
:102560000B0F04BF09010CF1040C8B0F04BF890091
:102570000CF1020CCB0F04BF49000CF1010CCCF1A3
:102580002003A0EB0C0022FA03F302FA0CF241EA5A
:10259000030100F10100704720F07F4C80EA030046
:1025A00023F07F47ACEB070303F57C5300F00040BA
:1025B00003F1FF032DE980494FEA154B09B44FEAB7
:1025C000144325EA0B4E24EA03480FF2042606EBD7
:1025D000132749083E785FEA320203FB0667C7F516
:1025E000000707FB06F64FEA54374FEAD64606F1D6
:1025F000020607FB066CCCF1005C4FEA1C472CEA94
:10260000074C07FB06F40CFB06F504EB15464FEAF6
:10261000961634BF00204FF000404FEAD13706FB3A
:1026200007FC4FEA1C4C0CFB0BF7D21B03FB0CF70F
:1026300061EB07010CFB0EF7B0EB074072EB1742A2
:102640000CFB08F734BFA2EB0742B2EB074261EB89
:1026500017414FEA0C444FEA910706FB07FC4FEA8B
:102660001C4C0CFB0BF7B0EBC74072EB573203FB73
:102670000CF734BFA2EBC742B2EBC74261EB573154
:102680000CFB0EF7B0EBC70072EB57720CFB08F7B0
:1026900034BFA2EBC702B2EBC70261EB5771039FD5
:1026A0004FEA816141EA921104EBCC044FEAD13741
:1026B0004FEA826206FB07FC42EA90124FEA806012
:1026C0004FEA1C4C0CFB0BF7D21B03FB0CF761EB26
:1026D00007010CFB0EF7B0EB074072EB17420CFB47
:1026E00008F734BFA2EB0742B2EB074261EB174198
:1026F0004FEA8C554FEA910704EB9C2406FB07FC3C
:102700004FEA1C4C0CFB0BF7B0EBC74072EB573297
:1027100003FB0CF734BFA2EBC742B2EBC74261EB3D
:1027200057310CFB0EF7B0EBC70072EB57720CFB86
:1027300008F734BFA2EBC702B2EBC70261EB5771D7
:1027400015EB4C254FEA816141EA92114FEA826212
:102750004FEAD13742EA901206FB07FC44F100042D
:102760004FEA80604FEA1C4C0CFB0BF7D21B03FBBB
:102770000CF761EB07010CFB0EF7B0EB074072EBB7
:1027800017420CFB08F734BFA2EB0742B2EB07423B
:1027900061EB174115EB1C154FEA813141EA92417B
:1027A0004FEA823242EA90424FEA80304FEA0C769A
:1027B00044F1000448EA03434EEA0B484FF0000E90
:1027C000B2EB080C71EB030724BF624639464EEBAF
:1027D0000E0E4FF0000B0018524149414BEB0B0B12
:1027E000B2EB080C71EB03077BF1000B24BF6246D0
:1027F00039464EEB0E0E4FF0000B00185241494186
:102800004BEB0B0BB2EB080C71EB03077BF1000BEE
:1028100024BF624639464EEB0E0E51EA020718BF3E
:1028200046F0010616EB0E7655F1000254F1000158
:1028300003D5BDE88901BDE80088BDE88901BDE890
:102840000048B619524141EB0101A3F10103704761
:1028500080807F7E7D7C7B7A7978777676757473DD
:10286000727171706F6E6E6D6C6C6B6A6A6968689C
:10287000676666656464636362616160605F5F5E32
:102880005E5D5D5C5C5B5B5A5A59595858575756A8
:10289000565555555454535352525251515050500D
:1028A0004F4F4F4E4E4D4D4D4C4C4C4B4B4B4A4A5F
:1028B0004A494949484848474747474646464545A3
:1028C00045444444444343434342424242414141DC
:1028D000002B26D4770021D01CB54FEA370703B46C
:1028E0004FF010004FF010014FF000000FBCBDE89A
:1028F00010400BF1010BBBF1010F08BF5FEA170796
:1029000022BF12F1010211F101014FF0004143F128
:10291000000300F0004043EA00007047F9D3570875
:10292000DAE746EA064613F1400F4FEA16461FDD86
:1029300013F1200FDFBF16430A46002120335B420C
:10294000C8D0C3F1200746EA064602FA07F74FEA65
:10295000164646EA0706C3F1200722FA03F201FAF7
:1029600007F721FA03F14FF0000342EA0702B1E74B
:1029700046EA020646EA06464FEA164646EA0106D7
:10298000BCBF46EA0646360C4FF000034FF000028B
:102990004FF000019EE72DE9C048934630B491E81E
:1029A000380007C831EA400C48BF34EA430C03D56D
:1029B000FFF7F2FDFFF78CFFF0BCBDE800882DE9C2
:1029C000C048934630B491E8380007C810F0804FF3
:1029D00008BF13F0804F03D100F005F8FFF778FF30
:1029E000F0BCBDE8008820F07F4780EA030023F0B8
:1029F0007F4C07EB0C03A3F57C5300F00040A3F1E0
:102A0000FE0392F0000F00F0B38095F0000F00F08D
:102A100077802DE901494FEA11404FEA144621EA37
:102A2000004800FB06FC24EA064708FB06F607FB05
:102A300008F800FB07F718EB06484CEB164C4FEA7A
:102A4000124B18EB07484FEA15464CEB174022EAA9
:102A50000B4E0BFB06FC25EA06470EFB06F607FBB2
:102A60000EFE0BFB07F71EEB064E4CEB164C4FF021
:102A700000061EEB074E4CEB174B18EB0B0840F112
:102A8000000018EB0E0B58EB000840F100008F1A05
:102A90004FF000013CBFC943661B14BFB5EB040CEB
:102AA00000213CBFC943F61B4FEA17444EEA8E0E85
:102AB00027EA04454FEA1C4704FB07622CEA074C4F
:102AC00005FB07F70CFB05F604FB0CFC16EB0746B1
:102AD00042EB174216EB0C4642EB1C421BEB060680
:102AE00058EB0202414146EA9E0601D5BDE8018944
:102AF000B619524141EB0101A3F10103BDE801897F
:102B00004FEA14454FEA114724EA054621EA074CEB
:102B100005FB07F406FB07F70CFB06F105FB0CFCB5
:102B200011EB074144EB17444FEA124711EB0C41FC
:102B300044EB1C4422EA074C05FB07F206FB07F7AF
:102B40000CFB06F605FB0CFC16EB074642EB1742A6
:102B500016EB0C4642EB1C456A1854F1000148BFC5
:102B60007047B619524141EB0101A3F101037047CF
:102B700095F0000F37D04FEA11424FEA144721EA8F
:102B8000024624EA074C02FB07F106FB07F70CFBA1
:102B900006F402FB0CFC14EB074441EB17414FEA2F
:102BA000154714EB0C4441EB1C4125EA074C02FB92
:102BB00007F506FB07F70CFB06F602FB0CFC16EB11
:102BC000074645EB174516EB0C4645EB1C42121920
:102BD00051F1000148BF7047B619524141EB010164
:102BE000A3F1010370474FEA14454FEA114724EA65
:102BF000054621EA074C05FB07F106FB07F70CFB2E
:102C000006F24FF0000605FB0CFC12EB074241EB0D
:102C1000174112EB0C4251EB1C4148BF7047921810
:102C200041EB0101A3F10103704710B507F0D5FC9A
:102C300007F0D2FCBDE8104007F0DCBB00210160CA
:102C4000C1607047FEE7000010B50146034802F07E
:102C500061F9024802F03EF9002010BDD0090020C1
:102C60000A46094910B5D1F81812D1F814120029F2
:102C70001CBF012010BD0146034802F051F9BDE818
:102C80001040014802F054B9D009002070470000FC
:102C9000002251B1012908BF4FF4807205D00229EA
:102CA0000CBF4FF400724FF440720E490B6823F4CE
:102CB00040730B600B681A430A600A6822F0F8023E
:102CC0000A600A68F82393FAA3F3B3FA83F39840EF
:102CD00040F0020010430860086840F4803008604B
:102CE00070470000103C02402049086810F0100FA7
:102CF0001F4805D0C26942F01002C26110220A606A
:102D00000A6812F0200F05D0C26942F00802C261C1
:102D100020220A600A6812F0400F05D0C26942F012
:102D20000402C26140220A600A6812F0800F05D0D6
:102D3000C26942F00202C26180220A600A6812F48B
:102D4000807F06D0C26942F00102C2614FF48072F6
:102D50000A600A6812F0020F08BF7047C26942F0A9
:102D60002002C26102200860704700000C3C024053
:102D70003409002070B5174904460020C86100F0EE
:102D8000D9F9154D0646286810F4803F0FD000BFD2
:102D9000B4F1FF3F07D024B100F0CCF9801BA04272
:102DA00001D9032070BD286810F4803FF0D1286855
:102DB00010F0010F1CBF0120286028684FF4F97142
:102DC00031EA00001CBF002070BDFFF78DFF01201D
:102DD00070BD0000340900200C3C024090F8351012
:102DE000022903D08021416501207047052180F828
:102DF00035100068016821F0010101600020704772
:102E000031B508F0A1F8044608F09EF80099001BBF
:102E100001EB4102C2EBC111B0EBC10FF4D338BDDD
:102E20000348016841F00041016000207047000044
:102E3000103C02402DE9F0472D4F81461546387E63
:102E400098460E46012804BF0220BDE8F087012005
:102E500038764CF25030FFF78DFF08BB254CB9F1A6
:102E6000000F21D0B9F1010F2AD02068B9F1020F6B
:102E700020F440702060206830D040F44070206022
:102E8000206840F0010020603560C6F8048000BF73
:102E90004CF25030FFF76EFF216821F001012160F4
:102EA00000213976BDE8F087206820F4407020606A
:102EB00020682060206840F0010020603570E7E75E
:102EC000206820F440702060206840F4807020600A
:102ED000206840F0010020603580D9E740F40070A0
:102EE0002060206840F0010020603560D0E70000DD
:102EF00034090020103C02400648006810F0004FE2
:102F000004BF01207047044904480160044901607E
:102F100000207047103C024023016745043C0240FA
:102F2000AB89EFCD2DE9F84F00227A4EDFF8E8E1CA
:102F300001274FF0030A4FF00F0800BF0B6807FA94
:102F400002F42340A3427DD1D1F804C0BCF1020FAA
:102F500018BFBCF1120F15D14FEAD20C00EB8C0553
:102F6000D5F820904FEA427C4FEADC6C08FA0CFB63
:102F700029EA0B09D1F810B00BFA0CFC4CEA090C49
:102F8000C5F820C0D0F800904FEA420C91F804B088
:102F90000AFA0CF50BF0030B29EA05090BFA0CFBF6
:102FA0004BEA0909C0F80090D1F80490B9F1010F7B
:102FB00018BFB9F1020F05D0B9F1110F18BFB9F15F
:102FC000120F18D1D0F80890D1F80CB029EA0509F1
:102FD0000BFA0CFB4BEA0909C0F80890D0F80490F2
:102FE00029EA040491F80490C9F3001909FA02F9D6
:102FF00049EA04044460C468AC438D6805FA0CFCDB
:103000004CEA040CC0F80CC0D1F804C01CF0805F7E
:1030100079D0D6F800C04CF4804CC6F800C0D6F881
:1030200000C00CF4804CCDF800C022F0030C0CF171
:10303000804C0CF5983CDCF808589407240F08FAEB
:1030400004F900E05FE025EA0905A0F18049B9F53F
:10305000003920D0A0F18049B9F5013908BF4FF0FF
:10306000010918D0A0F18049B9F5023908BF4FF025
:10307000020910D0A0F18049B9F5033908BF4FF01B
:10308000030908D0A0F18049B9F504390CBF4FF00D
:1030900004094FF0050909FA04F42C43CCF8084858
:1030A000DEF800C04C682CEA030C14F4803F18BF13
:1030B0004CEA030CCEF800C0184CD4F800C04D68A0
:1030C0002CEA030C15F4003F18BF4CEA030CC4F8BB
:1030D00000C0134CD4F800C04D682CEA030C15F462
:1030E000801F18BF4CEA030CC4F800C00D4CD4F884
:1030F00000C04D682CEA030C15F4001F18BF4CEA01
:10310000030CC4F800C0521C102AFFF417AFBDE82E
:10311000F88F000044380240003C0140043C01406C
:10312000083C01400C3C0140002A08BF09048161B1
:10313000704700000148006870470000E801002067
:1031400002480168491C016070470000E801002046
:103150000B4810B5016841F400710160016841F449
:1031600080610160016841F480710160032000F01A
:10317000A3F80F2000F006F800F05EF8002010BD64
:10318000003C024038B523480025016841F00801A1
:103190000160006800F0080000901F48016841F0DD
:1031A00008010160016821F00801016001F0DEFB07
:1031B0001B4C1A481C492060681EE06019480068D2
:1031C0002561B0FBF1F0401EC4E9010520466561B0
:1031D00001F0E6F81549322006F0A2FB14494FF43D
:1031E0008020C1F800010021204601F0F5F80421FB
:1031F000204601F0F1F82068416A0E4A116001F59D
:103200007A7181632068C16841F00401C1600020C7
:1032100038BD00004038024020380240000C004019
:10322000200400209801002040420F008DAE0008CD
:1032300004E000E094010020704700F01F0101222B
:1032400002FA01F14009800000F1E020C0F800110D
:1032500070470000174B10B41B68C3F30223C3F17F
:10326000070CBCF1040F88BF4FF0040C1C1D072C89
:1032700034BF0023DB1E012404FA0CFCACF1010C6A
:103280000CEA0101994004FA03F35B1E1A40114352
:1032900000284FEA0111A1BF00F1E02080F80014DE
:1032A00010BC704700F00F0000F1E02080F8141D02
:1032B00010BC70470CED00E0074900F007000A68F9
:1032C0004FF6FF031A4042EA002040F0FD7040F044
:1032D00080600860704700000CED00E0006841620B
:1032E0000020704770B400680023D0F824C0002983
:1032F00004BF4CEA0241816218D0846A0CEB144C82
:103300004C1E18BF4FF4827509D000BF05EB830631
:1033100086595B1CDBB20CEB164C9C42F6D84FF482
:10332000807303EB81014CEA0242425070BC0020E2
:103330007047D0F8B40301F046BFC1EBC10200EB07
:103340008202D0F8B403526C01F0B0BE2DE9F04710
:103350000E46074672B6012936D1234C214D402234
:10336000206805F5177105EB8010FDF7E4FB69781F
:10337000A878042202EB012100EB010860684FF0FD
:1033800000094FF0010A012810D12978284604F0DD
:10339000A1FC00281CBFC4F80490B8F1400F05DD63
:1033A000A8F101000AEBA010C5F874092068401CC0
:1033B0002060D5F87409401EC5F87409D5F8740961
:1033C000002808BFC4E9009AC6EBC60007EB8000DE
:1033D0003146D0F8E821D7F8B40301F0BFFE62B659
:1033E000BDE8F0874852002044030020D0F8B40321
:1033F00001F0EBBE10B5044601F07F03C3EBC30040
:103400000A4611F0800F04EB800014BF00F1380170
:1034100000F5EE710B70D009487094F88003012814
:1034200004BF022010BD012084F88003206802F050
:1034300093FA002084F8800310BD70B504460A4654
:1034400011F0800F01F07F0014BFC0EBC001C2EB90
:10345000C20104EB810114BF383101F5EE71002582
:103460008D700870D009487094F88003012804BF5B
:10347000022070BD012084F88003206802F04DFC1A
:1034800084F88053002070BD01F07F01C1EBC101C1
:1034900000EB8100B0F8F40180B2704770B50446CB
:1034A0008C4611F0800F01F07F00C0EBC00104EBEF
:1034B000810114BF383101F5EE7108705FEADC1C40
:1034C00081F801C08A60CB7018BFC8800025022B2C
:1034D00008BF0D7194F88003012804BF022070BD5D
:1034E000012084F88003206802F07AF9284684F8E5
:1034F000805370BD70B504468C4601F07F00C0EB70
:10350000C00104EB81010025C1F8E821C1E97C3547
:1035100081F8DD5181F8DC01206901F5EE710128A7
:1035200008BF0A6194F88003012804BF022070BD1F
:10353000012084F88003227C20681CF07F0F05D0D6
:1035400002F050FC84F88053002070BD02F01AFB9A
:10355000F8E770B504460D4611F0800F01F07F00CA
:1035600014BFC0EBC001C5EBC50104EB810114BF62
:10357000383101F5EE7101228A700870E80948704F
:1035800094F88003012804BF022070BD84F88023D2
:10359000206802F0F4FB15F07F0F05D1217C04F5C3
:1035A0006172206802F09AFB002084F8800370BDED
:1035B00070B504468C4601F07F00C0EBC00104EBFF
:1035C000810100254A64C1E91335012381F83930AE
:1035D00001F8380F2069012808BF0A6194F88003B8
:1035E000012804BF022070BD84F88033227C20684B
:1035F0001CF07F0F06D002F0F5FB00BF84F880536B
:10360000002070BD02F0BEFAF8E700002DE9F04F8F
:103610000568044683B00026284602F054FD0028C1
:103620001CBF03B0BDE8F08F206802F075FD0028D4
:1036300004BF03B0BDE8F08F206802F06DFD10F00C
:10364000020F04D02068416901F002014161206845
:1036500002F062FD10F4002F4FF008084FF0100A3E
:103660004FF0010B4ED0206802F038FD070049D022
:1036700017F0010F43D0F1B2206802F045FD8146FA
:1036800010F0010F2AD005EB4611C1F808BB2069E4
:10369000012811D1C6EBC60004EB8000D1F8101B45
:1036A000D0F8E421C1F31201511AC0F8F411D0F896
:1036B000E8111144C0F8E811F1B22046FFF746FEC8
:1036C0002069012802BF002ED4F8F001002805D19E
:1036D00004F561720121206802F000FB19F0080F67
:1036E00006D0204600F0DDFA05EB4610C0F8088B46
:1036F00019F0100F1CBF05EB4610C0F808AB761C84
:103700007F08B5D1206802F007FD10F4802F75D036
:10371000206802F0DCFC5FEA00094FF000066DD083
:1037200019F0010F6BD0F1B2206802F0DEFC074601
:1037300010F0010F28D00121D5F8342801FA06F045
:1037400022EA0000C5F8340805EB4610C0F8081955
:103750002069012807D1C6EBC60004EB8000D0E940
:10376000102111444164F1B22046FFF7E6FD2069C3
:10377000012802BF002EE06C002805D104F561721B
:103780000121206802F0AAFA17F0080F04D005EB17
:1037900046110820C1F8080917F0100F04D005EBF6
:1037A00046111020C1F8080917F0400F04D005EBAE
:1037B00046114020C1F8080917F0020F04D005EBAC
:1037C00046110220C1F8080917F0800F49D020687F
:1037D0000190C6EBC60004EB800000F13808D8E980
:1037E0000501471AD8F80800874288BF0746F81C29
:1037F0004FEA900A019800EB461B1DE036E030E0EE
:10380000471AD8F80800B84238BF0746F81C4FEAF4
:10381000900A207C0090BBB2F2B2D8F80C1001984C
:1038200002F0C4FCD8F80C003844C8F80C00D8F8F2
:1038300018003844C8F81800DBF8180980B2504561
:1038400084BFD8E90501884201D90028D8D147B9F9
:1038500001990120B040D1F8341881430198C0F893
:103860003418761C5FEA59097FF45AAF206802F0D9
:1038700053FC10F0004F0DD0D5F8040820F00100E3
:10388000C5F80408204600F0F2F92068416901F00B
:1038900000414161206802F03FFC10F4006F0CD041
:1038A000D5F8080810F0010F1CBF204600F016FAEA
:1038B0002068416901F400614161206802F02CFC3C
:1038C00010F4805F5CD0D5F8040820F00100C5F842
:1038D00004080021206802F0C5FB6068D0B110F038
:1038E00001004FF0FF021CBFC5F80829C5F8082BDE
:1038F000616881420ED900BF05EB4011C1F808296B
:10390000C1F8082BC1F82829C1F8282B6168801C50
:103910008142F1D84FF0FF30C5F81808D5F81C08DF
:1039200040F00110C5F81C08206B60B1D5F8840880
:1039300040F00B00C5F88408D5F8440840F00B00AF
:10394000C5F844080BE0D5F8140840F00B00C5F8A2
:103950001408D5F8100840F00B00C5F81008D5F889
:10396000000820F4FE60C5F80008217C04F56172AF
:10397000206802F0B3F92068416901F48051416187
:10398000206802F0C9FB10F4005F1CD0206801F031
:103990006FFF2068C16821F47051C160206802F097
:1039A00075FB60B30320E060402060612068C1685F
:1039B00041F4C051C160204600F048F920684169D7
:1039C00001F400514161206802F0A6FB10F0100FD5
:1039D00041D02068816921F010018161D5F82080F3
:1039E00008F00F00C0EBC00004EB800000F5EE779C
:1039F000C8F3434002280CD006281CD026E0002043
:103A0000E0604FF4007060612068C16841F41051BB
:103A1000D0E747F6F07018EA000F17D0C8F30A1283
:103A200090462846F96802F07BFBF8684044F8604D
:103A3000B869404409E0082204F56171284602F0A3
:103A40006FFBB869C8F30A110844B861206881693E
:103A500041F010018161206802F05EFB10F0080F58
:103A600007D0204600F007F92068416901F00801FD
:103A70004161206802F050FB10F4801F08D0F1B2C1
:103A8000204600F03AF82068416901F48011416154
:103A9000206802F041FB10F4001F08D0F1B220466C
:103AA00000F02FF82068416901F40011416120689D
:103AB00002F032FB10F0804F07D02046FFF739FCB0
:103AC0002068416901F080414161206802F024FBD7
:103AD00010F0040F04BF03B0BDE8F08F2068456804
:103AE00015F0040F1CBF2046FFF780FC20684168DA
:103AF0002943416003B0BDE8F08FD0F8B40301F072
:103B0000B5BBD0F8B40301F0B3BB002804BF01205B
:103B100070472DE9F04104468AB0032084F8810300
:103B2000204600F05DF8206802F026F81034B4E872
:103B3000EF108DE8EF1074E80C01CDE9080194E86E
:103B40000F0001F0AFFE0021206802F006FB00220A
:103B50000F2101251046C2EBC20304EB8303491E6B
:103B600083F8395083F83820DA8783F83B001864EB
:103B70005864D86402F10102EDD14FF48273C1EBB5
:103B8000C10204EB820203EB810C82F8DD0182F8B2
:103B9000DC11D18782F8DF01C2F8E401C2F8E80144
:103BA000C2F8F001226842F80C00491C0F29E6D344
:103BB00004F1100090E8CF118DE8CF11D4E90C0189
:103BC000CDE9080194E80F0001F01CFF84F881534F
:103BD000206801F00BFF0AB00020BDE8F081000072
:103BE00000B5006887B0B0F1A04F1CBF07B000BDA2
:103BF0004FF4C0500090022001900020029003205A
:103C000003900A20049069460D48FFF78BF90D4890
:103C1000016841F0800101600B48016841F4804176
:103C200001600068002200F48040059011464320A6
:103C3000FFF710FB4320FFF700FB07B000BD0000BB
:103C400000000240343802404438024010B50446B7
:103C5000C0680121002808BF0021D4F8B40301F096
:103C60004CFBD4F8B403BDE8104001F014BBD0F80D
:103C7000B40301F02FBBD0F8B40301F031BB10B591
:103C8000044690F88003012804BF022010BD0120E3
:103C900084F88003206802F077FA002084F880031B
:103CA00010BDD0F8B42300F56171104601F02FBBB0
:103CB00010B5044690F88003012804BF022010BD0F
:103CC000012084F88003206801F084FE206802F05F
:103CD000C3F9002084F8800310BD000010B504462D
:103CE000D0F8B40301F050FB2068D0F8001E41F07A
:103CF0000101C0F8001E206A002808BF10BD03485B
:103D0000016841F00601016010BD000010ED00E007
:103D10002DE9F05F5F4F06468946386801F0FF0ADB
:103D200000F00F00484506D287F800A0386800F080
:103D30000F00484540D13078574D10F0020F05D0A4
:103D40002868B16820F0F00008432860307810F04F
:103D5000010F65D070685149012825D0022818BF8D
:103D60000328096825D011F0020F65D0296821F0D9
:103D7000030108432860FFF7DDF90446706841F24B
:103D80008838012819D0022827D00328286834D081
:103D900010F00C0F44D000BFFFF7CCF9001B4045DA
:103DA0003AD90320BDE8F09F096811F4003FDDD146
:103DB00042E011F0007FD9D13EE0286800F00C000D
:103DC00004282DD0FFF7B6F9001B4045E9D8286834
:103DD00000F00C000428F5D122E0286800F00C0067
:103DE00008281DD0FFF7A6F9001B4045D9D8286840
:103DF00000F00C000828F5D112E04FF00C0B3BEA64
:103E000000000DD0FFF796F9001B4045C9D828687F
:103E10003BEA0000F6D103E0286810F00C0FBBD19C
:103E2000386800F00F00814509D287F800A0386893
:103E300000F00F00484502D00120BDE8F09F307827
:103E400010F0040F05D02868F16820F4E050084312
:103E50002860307810F0080F06D02868316920F407
:103E6000604040EAC100286000F04EF82968F02266
:103E700092FAA2F201F0F001B2FA82F2D140084ABD
:103E8000515CC840074908600F20FFF77BF900200C
:103E9000BDE8F09F003C0240083802400038024074
:103EA00098B200089801002008480949006809688C
:103EB0004FF4E05292FAA2F201F4E051B2FA82F227
:103EC000D140044A515CC84070470000980100206E
:103ED0000838024098B20008084809490068096893
:103EE0004FF4604292FAA2F201F46041B2FA82F217
:103EF000D140044A515CC84070470000980100203E
:103F00000838024098B200082048006810F00C0100
:103F10001F4808BF7047DFF87CC0042904BF604613
:103F20007047082918BF704710B41B4B196801F07F
:103F30003F02196811F4800F47F6C0710BD0BCFB2B
:103F4000F2F01A680A4091FAA1F1B1FA81F122FA6D
:103F500001F148430AE0B0FBF2F01A680A4091FA16
:103F6000A1F1B1FA81F122FA01F1484319684FF445
:103F7000403292FAA2F201F44031B2FA82F2D14018
:103F8000491C4900B0FBF1F010BC704708380240F2
:103F90000024F4000048E801043802402DE9F84FFD
:103FA00004460078CE4FCF4D10F0010F40D0386856
:103FB00000F00C00042809D0386800F00C00082834
:103FC0000DD1281D006810F4800F08D0286810F467
:103FD000003F2DD06068002800F07F8128E0C249B2
:103FE00020790870606890B1FFF7A4F80646286849
:103FF00010F4003F1CD100BFFFF79CF8801BC828BD
:1040000000F21581286810F4003FF5D010E0FFF7AA
:1040100091F80646286810F4003F09D0FFF78AF8A7
:10402000801BC82800F20381286810F4003FF5D1F6
:104030002078DFF8B88210F0020F4FF0000958D056
:1040400038684FF0F80A10F00C0F16D0386800F0FE
:104050000C00082804D1A648006810F4800F0CD08A
:10406000E06890B30120C8F80000FFF763F8064647
:10407000286810F0020F13D01BE0286810F0020F20
:104080001CBFE068012840F0288128689AFAAAF14C
:1040900020F0F8022069B1FA81F18840104312E063
:1040A000FFF748F8801B02287ED8286810F0020F1E
:1040B000F6D028689AFAAAF220F0F8012069B2FA3C
:1040C00082F290400843286013E0FFE7C8F80090B0
:1040D000FFF730F80646286810F0020F09D000BF3D
:1040E000FFF728F8801B02285ED8286810F0020F1E
:1040F000F6D1207810F0080F2ED07E48DFF8F8A116
:104100006169A1B101210160FFF714F80646DAF8F0
:10411000000010F0020F1FD1FFF70CF8801B0228DF
:1041200042D8DAF8000010F0020FF5D014E0C0F821
:104130000090FEF7FFFF0646DAF8000010F0020FCD
:104140000AD000BFFEF7F6FF801B02286FD8DAF80E
:10415000000010F0020FF5D1207810F0040F4FD0BE
:104160006648016841F0805101600068DFF890A165
:1041700000F080500090DAF8000040F48070CAF837
:104180000000FEF7D7FF0646DAF8000010F4807F43
:104190000CD100BFFEF7CEFF801B022847D8DAF80B
:1041A000000010F4807F00E041E0F3D0554E207A0B
:1041B0003070A06841F2883B88B1FEF7BBFF8246B1
:1041C000306810F0020F1BD1FEF7B4FFA0EB0A001D
:1041D00058452CD8306810F0020FF5D010E0FEF7EB
:1041E000A9FF8246306810F0020F09D0FEF7A2FF47
:1041F000A0EB0A0058451AD8306810F0020FF5D12C
:10420000A069E8B3396801F00C01082965D00228DB
:10421000C8F860900ED0FEF78DFF0446286810F0B5
:10422000007F57D0FEF786FF001B02284ED90320DF
:10423000BDE8F88FFEF77EFF0646286810F0007F85
:1042400009D000BFFEF776FF801B0228EFD8286850
:1042500010F0007FF6D1D4E90701014347F6C072A0
:1042600092FAA2F2606AB2FA82F29040A26A4FF029
:10427000FF3303EB52024FF4403393FAA3F300E011
:1042800028E0B3FA83F39A40104308434FF070627A
:1042900092FAA2F2E16AB2FA82F291400143144822
:1042A00001600120C8F86000FEF744FF044628685A
:1042B00010F0007F0ED100BFFEF73CFF001B02286C
:1042C000B5D8286810F0007FF6D003E0286810F019
:1042D000007FA7D10020BDE8F88F0120BDE8F88F4E
:1042E00008380240003802400238024000004742CD
:1042F00004380240800E4742743802404038024081
:104300000070004070380240002804BF0120704750
:1043100070B5044690F85100002520B984F850503B
:10432000204600F037F8022084F851002068016828
:1043300021F040010160D4E901010843D4E90312EE
:104340001143084361690843218B01F4007108435C
:10435000E1690843216A0843A16A084321680860AB
:10436000A069042101EA1040616A0843216848609D
:10437000A06AB0F5005F02D12168E06A0861206898
:10438000C16921F40061C1616565012084F85100B3
:10439000002070BD7047704710B5FFF7FCFF10BDDF
:1043A000002804BF0120704710B5044690F839007A
:1043B00028B9002084F83800204600F00CF80220CC
:1043C00084F83900211D206800F090FB012084F85A
:1043D0003900002010BD70470268012303FA01F183
:1043E000136A8B431362136A194311620168A1F1C6
:1043F0008042B2F5803203D14A6C42F400424A64F2
:104400000068016841F00101016000207047006808
:1044100081B0016811F0010F04BF016811F0020FB3
:1044200003D04068009001B07047016811F0040F9C
:1044300004BF016811F0080FF3D101B0704700000C
:1044400070B5016804460868CA684B6910F00F0F20
:104450004FF0200543D040F2011C13EA0C0F00F08E
:10446000F18010F0010F18BF12F4807F05D0D4F84E
:104470003CC04CF0010CC4F83CC010F0040F18BF55
:1044800013F0010F05D0D4F83CC04CF0020CC4F876
:104490003CC010F0020F18BF13F0010F05D0D4F884
:1044A0003CC04CF0040CC4F83CC010F0080F18BF1E
:1044B00013F0010F03D0E36B43F00803E363E36BF6
:1044C000002B08BF70BD10F0200F18BF12F0200F96
:1044D00072D094F83A202046222A44D07CE010F092
:1044E000200F18BF12F0200F67D094F83A20204612
:1044F000222A18BF70BD8268B2F5805F1ED00269A3
:104500005AB3496801F07F02816A4B1C83620A70CA
:10451000C18D491E0904090CC18518BF70BD016811
:10452000CA6822F49072CA6001684A6922F00102E6
:104530004A6180F83A5000F0FDF870BD0369826A64
:104540004968002B14BFC9B2C1F308011180816A08
:1045500014BF491C891C8162DAE74A68816A4B1CD6
:1045600083620A70D4E78268B2F5805F0FD0026977
:10457000E2B1496801F07F02816A4B1C83620A70D4
:10458000C18D491E0904090CC18525D116E00369B6
:10459000826A4968002B14BFC9B2C1F308011180B7
:1045A000816A14BF491C891C8162E9E74A68816AF3
:1045B0004B1C83620A70E3E70EE043E00168CA68BF
:1045C00022F49072CA6001684A6922F001024A61CD
:1045D00080F83A5000F0AEF820684169E26BC1F310
:1045E000801102F00802114326D0C16821F49071B5
:1045F000C1602068416921F00101416184F83A50AD
:104600002068416911F0400F12D0416921F040014A
:104610004161606B60B12D490165606BFEF7DEFBA7
:10462000002808BF70BD606B016DBDE87040084791
:104630002046FFF7ECFE70BD2046FFF7E8FE0020A5
:10464000E06370BD10F0800F18BF12F0800F2CD007
:1046500094F83900212818BF70BDA068B0F5805FBC
:10466000206A16D0411C2162216800784860E08CE5
:10467000401E0004000CE08418BF70BD2068C168B3
:1046800021F08001C1602068C16841F04001C16033
:1046900070BD0088C0F30800486020690028206AC7
:1046A00014BF401C801C2062E1E710F0400F14BFD3
:1046B00012F0400F70BD2046CA6822F04002CA6066
:1046C00084F8395000F037F870BD0000814B0008C5
:1046D000002804BF0120704770B5044690F83900E7
:1046E000002520B984F83850204600F022F8242014
:1046F00084F839002068C16821F40051C160204667
:1047000000F046FA2068016921F4904101612068B7
:10471000416921F02A0141612068C16841F40051DA
:10472000C160E563202084F8390084F83A00002055
:1047300070BD704770470068016811F0400F1CBFE2
:104740006FF0400101607047FEE7000010B50022E5
:104750000849094800F084FC0849074800F038FE81
:104760000749054800F0CEFBBDE81040024800F0C4
:1047700043BE000050030020D0090020FC020020AE
:1047800034030020FEE770470148FEF73FBF0000FA
:10479000044C0020704770472DE9F04F394D93B01D
:1047A0000024286840F0805028602868364E00F0C9
:1047B00080501190306820F4404040F40040306058
:1047C00030684FF0010800F4404011900520CDE919
:1047D000008002277805CDE906704FF01009A82067
:1047E000CDE908904FF0040A0720CDE90AA06846F9
:1047F000FFF7D4FB4FF00F0B70B9A814CDE90E40B2
:10480000CDE90CB702210CA81094FFF781FA00281B
:1048100004BF13B0BDE8F08F286840F080502860D6
:10482000286800F080501190306820F4404040F437
:1048300000403060306800F4404011900320CDE922
:104840000004CDE90389CDE90674C020CDF820909D
:10485000CDF82CA0CDE909076846FFF79FFB78B992
:104860004FF48050CDE90E40CDE90CB702210CA8E1
:104870001094FFF74DFA002804BF13B0BDE8F08F85
:10488000FEE70000403802400070004038B50024C8
:10489000224908283CD2DFE800F0040D161F283B0F
:1048A0003B311F4C086840F001000860086800F0C8
:1048B00001002BE01B4C086840F00200086008680B
:1048C00000F0020022E0184C086840F00400086084
:1048D000086800F0040019E0144C086840F0080073
:1048E0000860086800F0080010E0114C086840F00B
:1048F00010000860086800F0100007E00D4C086820
:1049000040F080000860086800F08000009002E03D
:1049100009A005F081FA204638BD00003038024079
:10492000000002400004024000080240000C024067
:1049300000100240001C024050696E6D61702065DD
:1049400072726F723A2077726F6E6720706F727436
:10495000206E756D6265722E0000000010B5FEF7C6
:10496000EFFBBDE81040FFF717BD0000DFF86CC09B
:1049700030B4DCF800001A4B10F00C01194806D0D6
:104980005C00042908BF046002D008290CD0036031
:10499000DCF80010144AC1F30311515C026822FADA
:1049A00001F1016030BC704710490A68C2F38055BC
:1049B0000A68002D02F03F0214BFB4FBF2F2B3FB11
:1049C000F2F20B680968C3F388135A43C1F301413B
:1049D000491C4900B2FBF1F10160D9E708380240F7
:1049E0000024F4009801002044B20008043802407A
:1049F00030B5314887B0016841F4700101602F483B
:104A0000016841F0010101602D4A00211160026836
:104A100022F4102222F080720260031D294A1A60DB
:104A2000026822F480220260274801602749580664
:104A300008602849264808602748016821F00701D6
:104A40000160016841F001010160FEF781FB23482C
:104A5000016841F0010101600068214D00F0010092
:104A60000590012000900190029002200390694679
:104A70002846FEF757FA012211462846FEF754FB56
:104A8000184C0121491CA142FCDB002201212846CF
:104A9000FEF74AFB0220401CA042FCDBFFF77CFE35
:104AA0001148016841F008010160016821F0080126
:104AB000016007B030BD000088ED00E00038024022
:104AC00008380240103000240C38024008ED00E0A5
:104AD0000024F400980100200038014030380240E2
:104AE00000000240A08601002038024070B4026835
:104AF0001F4BDFF880C0204C204D984218BFB0F10A
:104B0000804F04D060451CBFA042A84203D14E682C
:104B100022F070023243984218BFB0F1804F14D097
:104B2000604518BFA04210D0A8421CBFA0F1804C25
:104B3000BCF5A03C09D0A0F1804CBCF5A23C1CBF48
:104B4000A0F1804CBCF5A43C05D1D1F80CC022F4F6
:104B500040724CEA020202608A68C2620A6882629B
:104B6000984204BF096901630121416170BC70472B
:104B7000000001400004004000080040000C00401C
:104B800010B5806B0021C185C184FFF740FC10BDCA
:104B90002DE9F041044600680169E26821F44051C2
:104BA000114301612068C1682369A268D4F81CC060
:104BB0001A43636921F4037143EA0C0321F414419D
:104BC0001A431143C16020684169A26921F4407110
:104BD00011434161E2693226B2F5004FBA48BB4940
:104BE000BB4D22685DD08A4218BF824240F01281DC
:104BF000FFF772F900EBC00101EB0010616889005A
:104C0000B0FBF1F7FFF768F900EBC00101EB001012
:104C100061688900B0FBF1F0A5FB001040096FF05E
:104C20001801484307EB800006EB0010A5FB0010BD
:104C3000400900F0F007FFF74FF900EBC00101EB6E
:104C4000001061688900B0FBF1F0A5FB001040097D
:104C500007EB0017FFF740F900EBC00101EB001074
:104C600061688900B0FBF1F8FFF736F900EBC0018D
:104C700001EB001061688900B0FBF1F0A5FB0010AA
:104C800040096FF01801484308EB800006EB001064
:104C9000A5FB00102168C0F3431038448860BDE8CC
:104CA000F0818A4218BF824259D1FFF715F900EB13
:104CB000C00101EB001061684900B0FBF1F0A5FBF9
:104CC000001040090701FFF707F900EBC00101EBF5
:104CD000001061684900B0FBF1F8FFF7FDF800EB48
:104CE000C00101EB001061684900B0FBF1F0A5FBC9
:104CF000001040096FF01801484308EB800006EBF4
:104D0000C000A5FB0010400900F0F80007EB4007C9
:104D1000FFF7E2F800EBC00101EB00106168490009
:104D2000B0FBF1F8FFF7D8F800EBC00101EB001081
:104D300061684900B0FBF1F0A5FB001040096FF07D
:104D40001801484308EB800006EBC000A5FB0010EB
:104D50002168C0F3421038448860BDE8F081FFF755
:104D6000A3F800EBC00101EB001061684900B0FB43
:104D7000F1F0A5FB001040090701FFF795F800EBE3
:104D8000C00101EB001061684900B0FBF1F8FFF7CA
:104D90008BF800EBC00101EB001061684900B0FB2B
:104DA000F1F0A5FB001040096FF01801484308EB33
:104DB000800006EBC000A5FB0010400900F0F800E1
:104DC00007EB4007FFF770F800EBC00101EB0010A4
:104DD00061684900B0FBF1F8FFF766F800EBC0012D
:104DE00001EB001061684900B0FBF1F0A5FB001079
:104DF00040096FF01801484308EB800006EBC00043
:104E0000A5FB00102168C0F3421038448860BDE85B
:104E1000F08100BFFFF748F800EBC00101EB001084
:104E200061688900B0FBF1F7FFF73EF800EBC001C5
:104E300001EB001061688900B0FBF1F0A5FB0010E8
:104E400040096FF01801484307EB800006EB0010A3
:104E5000A5FB0010400900F0F007FFF725F800EB74
:104E6000C00101EB001061688900B0FBF1F0A5FB07
:104E70000010400907EB0017FFF716F800EBC00120
:104E800001EB001061688900B0FBF1F8FFF70CF846
:104E900000EBC00101EB001061688900B0FBF1F08C
:104EA000A5FB001040096FF01801484308EB800093
:104EB00006EB0010A5FB00102168C0F34310384436
:104EC0008860BDE8F081000000140140001001403E
:104ED0001F85EB5110B5D0F81812002904BF02202D
:104EE00010BD027C002AD1F8042205D04023012104
:104EF00000F0CAF9002010BD4FF40073012100F04A
:104F0000C3F9F7E70246022000291CBF0020C2F8BF
:104F10001C127047D0F81802C0F804120020704725
:104F2000D0F81802C0F81022C0F80812002070470C
:104F300010B5D0F81812002904BF022010BDD1F816
:104F40001422002A1CBF012010BD0122C1F8142226
:104F5000B1F8102293B2D1F80822812100F01DFA95
:104F6000002010BD10B5D0F81422526890470020E0
:104F700010BD134610B50A46002100F085F9002047
:104F800010BD134610B50A46002100F006FA0020B5
:104F900010BD10B50323C0F80821C0F8F431C0F8E3
:104FA0000C2113460A46002100F06EF9002010BDC6
:104FB00010B505210023C0F8F4111A46194600F077
:104FC00063F9002010BD10B502238261C0F8F431EE
:104FD000C26113460A46002100F0DFF9002010BD2F
:104FE00010B504210023C0F8F4111A46194600F048
:104FF000D4F9002010BD000030B40025002804BF03
:1050000030BC7047034604784FF0000C44B100BF39
:1050100013F8014F0CF1010C0CF0FF0C002CF7D130
:10502000022303EB4C0313804B556A1C03238B5460
:105030000378AA1C002B12BF002330BC704700BFAE
:1050400010F801CB01F802C0521CD2B28B54521C92
:1050500090F800C0D2B2BCF1000FF1D130BC704763
:10506000002804BF02207047D0F81432002B1CBF68
:105070000023C0F81432002918BFC0F8101210B570
:10508000012180F8FC11027000F0AEF8002010BD84
:1050900010B5D0F82002FEF7D0F9002010BD10B5F1
:1050A000D0F82002FEF7A6F9002010BD70B5134617
:1050B000044659B1D4F814024269002A4CD094F83D
:1050C000FC01032804BF2046904745E0D4F8F411C2
:1050D000002504F11400022938D1D0E902218A42C6
:1050E0000DD9511A81608AB219462046FFF749FF4F
:1050F00000231A461946204600F0C6F826E040680C
:10510000B0FBF1F201FB12029AB9884211D3D4F834
:10511000F81188420DD2002211462046FFF731FFD8
:1051200000231A4619462046C4F8F85100F0ACF89E
:105130000CE0D4F81402C16829B194F8FC010328EA
:1051400004BF204688472046FFF732FF94F800024C
:10515000012808BF84F80052002070BD70B51546C4
:10516000044651B1D4F81402826952B394F8FC0198
:10517000032804BF2046904723E0D4F8F41104F537
:10518000827003291DD1D0E902C39C450CD9ACEB38
:1051900003038360C068984298BF03469AB22946C9
:1051A0002046FFF7E6FE0CE0D4F81402016929B1AD
:1051B00094F8FC01032804BF204688472046FFF7E7
:1051C0000FFF002070BD0020704710B5012180F84E
:1051D000FC11D0F81422017952689047002010BDCC
:1051E000D0F82002FEF750B910B50178002929D176
:1051F00015490222C1F8B403C0F820124FF0A040B4
:105200000860042048600020C1E90320C1E90502CC
:10521000C86108624862C86208630846FEF775FC08
:10522000002818BF01F05CFA80210748FEF756F805
:10523000402200210448FEF755F88022012102484F
:10524000FEF750F8002010BD044C002011F0800F34
:1052500001F07F01D0F82002C1EBC10100EB810019
:1052600014BF90F83A0090F8DE01704700207047B4
:105270000020704710B59C461346D0F820026246C5
:10528000FEF70CF9002010BD10B5D0F82002FEF793
:1052900031F9002010BD70B50022044640231146AC
:1052A000FFF7E8FF40252B46002280212046C4F866
:1052B0001051FFF7DFFF0120256284F8FC01D4F8CC
:1052C000180228B1D4F81402217942682046904788
:1052D000002070BD90F8FD1180F8FC11002070478F
:1052E00010B590F8FC11032905D1D0F81412C96942
:1052F000002918BF8847002010BD017400207047A6
:1053000010B5D0F82002FEF7BAFC002010BD10B591
:10531000044600F5027000F047F80120C4F8F401DB
:10532000B4F80E02C4F8F80194F8080210F01F0156
:105330000AD001290ED0022912D000F080012046A7
:1053400000F014F8002010BD04F50271204600F0B2
:1053500059F8F7E704F50271204600F020FAF1E76A
:1053600004F50271204600F095F9EBE710B5D0F88E
:105370002002FEF7EEF8002010BD10B5D0F8200294
:10538000FEF796FC002010BD90F8FC1180F8FD118E
:10539000042180F8FC110020704710B5D0F82002DD
:1053A000FEF706F9002010BD0A7802704A784270B4
:1053B0008A78CB7802EB032242800A794B7902EBA0
:1053C000032282808A79C97902EB0121C18070476A
:1053D00002460020002914BFC2F8141202207047B0
:1053E00010B5D0F81422022422B112689047002888
:1053F00008BF0024204610BD10B5FFF7BEFF0020F7
:1054000010BD0000F8B50D46497800260A2980F045
:10541000F180DFE801F0FAF9EFF8EF8505EFE3A49A
:1054200004466888010A082980F0C380DFE801F09B
:10543000C1040C1EC1C1555FD4F81012207C0A684B
:105440006946904701465DE0207C0028D4F81402AC
:1054500005D0C16A684688470146022051E0816A4A
:10546000684688470146022048704BE0C0B20628D3
:1054700074D2DFE800F0030B131B232BD4F81012B7
:10548000207C4A686946904701463BE0D4F81012F8
:10549000207C8A6869469047014633E0D4F81012B0
:1054A000207CCA686946904701462BE0D4F8101268
:1054B000207C0A6969469047014623E0D4F810121F
:1054C000207C4A696946904701461BE0D4F81012D7
:1054D000207C8A696946904707E0207C002868D1D3
:1054E000D4F81402416B6846884701460AE0207CE4
:1054F00000285ED1D4F81402016B68468847014643
:1055000007204870BDF8000000281CBFEA88002A68
:1055100057D0824288BF0246ADF8002020467AE08C
:105520000446A888002804BFE888002841D1A8784C
:1055300000F07F0594F8FC0103283AD084F8FE516E
:1055400029462046FFF7DCFE2046FFF749FD002DE7
:105550000CBF0120022084F8FC0132E029E0A97888
:105560004B4D04460129297023D894F8FC010228E8
:1055700002D003280ED01CE041B10320616084F802
:10558000FC012046FFF72CFF022812D02046FFF72F
:1055900027FD16E0B9B160688842F7D0C1B2204655
:1055A000FFF7E0FC297820466160FFF719FF022829
:1055B000ECD180212046FFF7D9FE00212046FFF7DD
:1055C000D5FE3046F8BD022084F8FC01204661601B
:1055D000FFF7C8FC2046FFF703FDF2E7E988012941
:1055E00008D190F8FC11022910D0032904BF012230
:1055F000011D10D004468021FFF7B8FE002120468F
:10560000FFF7B4FEDDE71BE02AE007E00021816040
:10561000012200F10801FFF7D6FCD2E790F8FC1157
:10562000022918BF0329E5D10121C160D0F8041275
:1056300000291CBF0321C160022200F10C01EAE72E
:105640000446688829460128BBD1C4F80402D4F86E
:1056500014028268204690472046FFF7C1FCB0E75D
:10566000044690F8FC012946022818BF0328A0D15F
:1056700048880128A5D10020C4F80402D4F81402F7
:105680008268204690472046FFF7AAFC99E7000071
:105690004C03002070B50D46044628780026097991
:1056A00000F06000202807D06878002848D0012842
:1056B00028D0032808D051E0D4F814022946826883
:1056C00020469047002070BD94F8FC01022802D0CB
:1056D000032805D03AE0002918BF802943D13DE0D6
:1056E000688828B900291EBF80292046FFF73EFEA2
:1056F000D4F8140229468268204690472046FFF7D6
:105700006FFC2BE094F8FC01022802D0032805D09E
:105710001CE0002918BF802925D11FE06888E8B95E
:1057200011F07F0F08D02046FFF7B2FCD4F8140226
:1057300029468268204690472046FFF751FC0DE03D
:1057400094F8FC0102280BD0032810D080212046B9
:10575000FFF70CFE00212046FFF708FE304670BD23
:1057600011F07F0FFAD02046FFF700FEF6E701F0B8
:105770007F0011F0800F04EB001014BF00F114053E
:1057800000F582752046FFF761FD002818BF012053
:105790000222286029462046FFF715FCDEE770B597
:1057A000044690F8FC010D4603280ED12879012803
:1057B0000BD8D4F81402826820469047E888002865
:1057C00004BF2046FFF70CFC07E080212046FFF7CE
:1057D000CDFD00212046FFF7C9FD002070BD00006F
:1057E0004B78012291F800C002FA0CF2012BD0F89C
:1057F0001C380CD043EA0242C0F81C280A7800EB9F
:105800004210D0F8002B12F4004F20D02CE092B2BE
:105810001A43C0F81C280A7800EB4210D0F800396F
:1058200013F4004F20D1D0F80039B1F808C0CCF300
:105830000A0C43EA0C03C978890441EA82511943EE
:1058400041F4004141F08051C0F800190CE0D0F85B
:10585000002B0B89C3F30A031A43C978034B43EAAD
:1058600081411143C0F8001B0020704700800010E8
:10587000D0F800196FF30A01C0F80019D0F8081821
:1058800001F00601042905D1D0F8001941F0030107
:10589000C0F80019D0F8041841F48071C0F8041859
:1058A000002070472B4ADDF800C0029B0999012BAC
:1058B00005D0C16841F04001C16001232DE0836B38
:1058C00023F480338363C36823F0400323F4840309
:1058D000C360C36823F44013C360012903D1C168C6
:1058E00041F48011C160012102E0491C914228D895
:1058F000036913F0004FF8D0016941F00101016123
:10590000012302E05B1C93421BD8016911F0010FD7
:1059100017D0F7E75B1C934210D8016911F0004FD4
:10592000F8D0016941F001010161012102E0491C47
:10593000914203D8036913F0010FF8D14FF480317D
:105940008163BCF1010F03D1816841F020018160C6
:1059500000207047400D030091F801C001220B7830
:1059600002FA03F3BCF1010FD0F83CC818D02CEABE
:105970000343C0F83C38D0F81C3891F800C002FA54
:105980000CF223EA0242C0F81C28097800EB41100F
:10599000D0F8001B21F40041C0F8001B0020704724
:1059A0009BB22CEA0303C0F83C38D0F81C3891F8BD
:1059B00000C002FA0CF292B223EA0202C0F81C28DC
:1059C000097800EB4110D0F8001921F40041C0F82B
:1059D0000019E3E710B5D0F8041821F00201C0F86F
:1059E00004180320FDF70CFA002010BD10B5D0F804
:1059F000041841F00201C0F804180320FDF700FA72
:105A0000002010BD2DE9F003DDE908280D9F069E5A
:105A1000D0F838C04CF4002CC0F838C02FB9D0F8FA
:105A200038C04CF4001CC0F838C04FF0000CC0F86F
:105A300000CED0F80048C0F80048012A0CD0D0F8B9
:105A4000002842F00302C0F8002800BF4FF484622F
:105A500002610123454A0BE0002BD0F8002818BF53
:105A600042F00102C0F80028F0E75B1C934203D823
:105A7000046914F0200FF8D110230361012302E020
:105A80005B1C934203D8046914F0100FF8D1C0F8DE
:105A900010C8C0F814C84FF0FF32C0F81828C0F87A
:105AA0001CC800224FF09045FF24002912D900BFE6
:105AB00000EB4213D3F8009919F0004F14BFC3F85C
:105AC0000059C3F800C9C3F810C9C3F80849521CEB
:105AD0009142EDD80022002912D900BF00EB4213F9
:105AE000D3F8009B19F0004F14BFC3F8005BC3F854
:105AF00000CBC3F810CBC3F8084B521C9142EDD831
:105B0000D0F8101821F48071C0F81018012E0CD1B3
:105B10001749C0F83018D0F8301841F0030141F4AB
:105B20008031C0F83018D0F83018C0F818C06FF0C5
:105B3000804141611EB9816941F010018161816933
:105B40000C4A11438161B8F1000F03D0816941F023
:105B500008018161012F05D1816941F0040141F003
:105B6000804181610020BDE8F0037047400D0300D3
:105B70000001800000383C80816821F001018160D3
:105B80000020704710B491F801C00B7800EB43136C
:105B9000BCF1010F2BD0D3F810CB6FF3120CC3F86C
:105BA00010CB0B7800EB4313D3F810CB6FF3DC4C26
:105BB000C3F810CB4B69002B1CBF8B684B610B7873
:105BC00000EB4313D3F810CB4CF4002CC3F810CBEC
:105BD0000B7800EB4313D3F810CB8C68C4F312049A
:105BE0004CEA040CC3F810CB012A6BD164E0D1F865
:105BF00014C0BCF1000FD3F810C941D06FF3120CE0
:105C0000C3F810C90B7800EB4313D3F810C96FF336
:105C1000DC4CC3F810C9D1F814C08B689C4598BF00
:105C200063464B610B7800EB4313D3F810C94CF477
:105C3000002CC3F810C90B7800EB4313D3F810C93C
:105C40004C69C4F312044CEA040C00BFC3F810C939
:105C5000012A2AD04A694AB1D0F834280B784FF08B
:105C6000010C0CFA03F31A43C0F83428097800EB4E
:105C70004110D0F8001941F00441C0F800192AE0A1
:105C80006FF3DC4CC3F810C90B7800EB4313D3F867
:105C900010C94CF4002CC3F810C90B7800EB431367
:105CA000D3F810C96FF3120CD0E70B7800EB431355
:105CB0000A69C3F81429D9E70B7800EB4313CA68C3
:105CC000C3F8142B097800EB4110D0F8001B41F009
:105CD0000441C0F8001B002010BC70470023C0F82E
:105CE000103BD0F8103B43F40023C0F8103BD0F831
:105CF000103B43F01803C0F8103BD0F8103B43F0C2
:105D0000C043C0F8103B012905D1C0F8142B4FF057
:105D10008021C0F8001B002070474B780A7800EB08
:105D20004212012B0BD0D2F8003B23F40013C2F82F
:105D3000003BCA78032A18BF022A15D01DE0D2F80A
:105D4000003923F40013C2F80039CA78032A18BFB7
:105D5000022A12D1097800EB4110D0F8001941F065
:105D60008051C0F8001908E0097800EB4110D0F824
:105D7000001B41F08051C0F8001B002070474B7899
:105D80000A7800EB4212012B05D0D2F8003B13F049
:105D9000004F15D01AE0D2F8003913F0004F05D1AA
:105DA000D2F8003923F08043C2F80039097800EBBB
:105DB0004110D0F8001941F40011C0F800190EE0AC
:105DC000D2F8003B23F08043C2F8003B097800EB97
:105DD0004110D0F8001B41F40011C0F8001B002056
:105DE0007047000030B44C786FF0604C0B7800EBDB
:105DF0004313012C32D0D3F8104B6FF31204C3F8C5
:105E0000104B0B7800EB4313D3F8104B6FF3DC44CB
:105E1000C3F8104B4B69002B7ED08C6823445B1E6B
:105E2000B3FBF4F39BB20C7800EB4414D4F8105B92
:105E30000CEAC34C45EA0C0CC4F810CB91F800C036
:105E400000EB4C1CDCF8104B8D686B43C3F3120362
:105E50002343CCF8103B012A7ED1D7E04C697CB3B8
:105E6000D3F810496FF31204C3F810490B7800EB14
:105E70004313D3F810496FF3DC44C3F810494C695D
:105E80008B681C44641EB4FBF3F30CEAC34C0B7820
:105E900000EB4313D3F810494CEA040CC3F810C9C3
:105EA0000B7800EB4313D3F810C94C69C4F3120408
:105EB0004CEA040CC3F810C9CB78012B18D029E0A8
:105EC000FFE7D3F810C96FF3DC4CC3F810C90B78A7
:105ED00000EB4313D3F810C94CF4002CC3F810C9DD
:105EE0000B7800EB4313D3F810C96FF3120C0FE0DB
:105EF0000B7800EB4313D3F810C92CF0C04CC3F857
:105F000010C90B7800EB4313D3F810C94CF0005CB8
:105F1000C3F810C9012A00E062E021D0CB78012B40
:105F200026D04B696BB1D0F8343891F800C0012409
:105F300004FA0CFC43EA0C03C0F83438CB78012B8C
:105F400016D00B7800EB4313D3F800C94CF0044C87
:105F5000C3F800C9CB7800E05EE0012B68D118E0FF
:105F600091F800C000EB4C1C0B69CCF81439E5E744
:105F7000D0F8083813F4807F0B7800EB4313D3F884
:105F800000C90CBF4CF0005C4CF0805CC3F800C949
:105F9000D7E791F800C0CB68898A89B2FAB9C91CE1
:105FA0008A0845D012F0010106D053F8045B00EBDB
:105FB0000C3404F58054256091423CBF00EB0C305A
:105FC00000F5805034D200BF53F804CBC0F800C0B5
:105FD00053F804CBC0F800C0891C9142F4D327E0E9
:105FE0000B7800EB4313D3F810CB8C68C4F3120486
:105FF0004CEA040CC3F810CB0B7800EB4313D3F836
:1060000010CB4CF4002CC3F810CB24E70B7800EB3A
:106010004313CA68C3F8142BCA78012A0BD0097835
:1060200000EB4110D0F8001B41F00441C0F8001B08
:10603000002030BC7047D0F8082812F4807F0A781E
:1060400000EB4212D2F8003B14BF43F0805343F000
:106050000053C2F8003BE2E7816841F00101816032
:10606000002070470022202343EA81110161064984
:10607000521C8A4201D903207047036913F0200F94
:10608000F6D1002070470000400D03000021D0F839
:10609000082812F0060F14D0D0F8082802F00602E3
:1060A000022A0DD0D0F80828062333EA020207D0CE
:1060B000D0F8080800F00600042808BF022100E01C
:1060C000032108467047406900F001007047D0F88E
:1060D0001818D0F81C08084080B27047D0F818187B
:1060E000D0F81C080840000C7047D0F81028D0F8F1
:1060F0003438CB4003F0010342EAC31200EB4110F5
:10610000D0F808091040704700EB4111D1F8081B86
:10611000D0F814080840704741698069084070470A
:106120000346D01C820816D012F0010003F58053FC
:1061300003D0D3F800C041F804CB90420BD200BF8B
:10614000D3F800C041F804CBD3F800C041F804CB29
:10615000801C9042F4D30846704710B5C26822F004
:10616000C042C260012904BFC16841F0005105D09E
:10617000002904BFC16841F0804100D1C1603220D4
:10618000FCF73EFE002010BDD0F8002822F4FE628D
:10619000C0F80028D0F800284FF4FE6303EA01118C
:1061A0001143C0F80018002070470000DDF800C05F
:1061B000BCF1000F19D1DB1C5FEA930C15D01CF069
:1061C000010300EB023000F5805002D051F8042B9F
:1061D0000260634509D200BF51F8042B026051F8F8
:1061E000042B02609B1C6345F6D300207047FEE73A
:1061F00070B50C460546FCF77FFE084AF321116096
:1062000002210420FCF744FD0023224629461846BB
:10621000FCF710FEBDE87040FCF702BE0C3C0240EB
:10622000002A18BFB0F5A37F24BF4FF0FF3070479E
:1062300070B50E460D4900EB4000154651F8204060
:1062400060B2B0F1FF3F07D0094804F0030200211B
:106250000260084803F05CFAC4F307212B4632467B
:10626000044803F009F8002070BD000004B30008E2
:106270000C040020A05C0020002A18BFB0F5A37F0A
:1062800024BF4FF0FF30704770B50E46114900EB48
:10629000400001EB8000154604688088C0F30720A9
:1062A000012804BF4FF0FF3070BD60B2B0F1FF3F76
:1062B00007D0094804F0030200210260074803F0F8
:1062C00027FAC4F307212B463246044803F092F81C
:1062D000002070BD04B300080C040020A05C002066
:1062E00010B5002204490548FEF71AFE0449034888
:1062F000FEF710FE002010BDFC2B0020D00900206E
:10630000F40B002010B5054803F02AF900221146CD
:10631000024803F0FDF9002010BD0000A05C002041
:1063200010B1102800D811B94FF0FF3070472DE997
:10633000F04F89462DED048BD1B080464FF4887123
:1063400002A8FAF76FFC0026B8F1000F7EDDDFF837
:1063500058B3F5EE008A9FEDD59A10279FEDD48AA9
:10636000C6EB061000EB800009EB8004052202A9B1
:106370000B20FFF755FF9DF80800002869D0102872
:1063800067D89DF80C5065859DF80BA005F11002AB
:1063900002A90420FFF744FF2A4602A904F12C00B9
:1063A000FAF70EFC02A9485D20710A2851D2C14AB1
:1063B000135C1BF80000C04A207394F804C052F824
:1063C0002020BE4850F82C00104420604819227B41
:1063D0004179112B00EE101AB94901EB8201B8EE98
:1063E000400AD1ED000A30EE200A84ED060A18BFFB
:1063F000102B34D0202B00F02581002161716173B6
:1064000084ED068A84ED078A84ED088A84ED098A82
:10641000A173216121758379C27990F809C003EBDA
:106420000222037A1B0403EB0C631A44521AA54997
:1064300089691144A160817AC07A01EB002020852E
:1064400000210B2001F09EF8761C00E001E046459B
:1064500086DB51B03046BDEC048BBDE8F08F0AF00E
:10646000070101293ED0052908BF677137D00729E8
:1064700014BF00211121617118BF4FF0000E2ED002
:10648000677390F90210112B00EE101AB8EEC00AD3
:1064900020EE280A84ED070A90F9031000EE101A86
:1064A000B8EEC00A20EE280A84ED080A90F904101C
:1064B00000EE101AB8EEC00A20EE280A84ED090A90
:1064C0000EBF032180498978A17341780909CA1F49
:1064D000062A78D2DFE802F00B0D0F1113154FF0EA
:1064E000010ECDE7012161714FF0000EC8E70222D5
:1064F00008E0042206E0082204E0276103E02022ED
:1065000000E0402222614278C2F3420CBCF1010F4C
:1065100008BF012259D0BCF1020F08BF022254D09B
:10652000BCF1030F08BF03224FD0BCF1040F1ABF08
:1065300000222275042248D0A27B032A47D0022AD7
:1065400004BF2269402A47D000224D92102B45D02B
:10655000722200925FF00102A1F1060ABAF1060F61
:1065600064D8002A62D005EB4E05C1EB450ACDF890
:106570001CA11AF1070F48D04D1CA1F1010A05FA20
:106580000AF5DDF834A1A1F1040ECAF1040A0AFAF1
:106590000EFA5544B5FBF2FE479D07EB8C0C05F156
:1065A000060A4D9D6D4201EB4501BAFBF1F501FB79
:1065B00015A1491C01FB0CF1B1FBF2F1009A7244E8
:1065C000114434E0FFE700229CE72275B4E722691A
:1065D000202A18BF402AB7D10122B6E73A4A92785A
:1065E000012A0ED0022A08D0032A0CBF4022002222
:1065F00000920CBF01220022AEE72022009202226C
:10660000AAE7102200920422A6E701F1010CA1F1F1
:10661000010A0CFA0AFC4FF0030A091F0AFA01F1F9
:106620006144B1FBF2FEA901A031C5E70021112BA5
:106630007FF4F1AE94ED060A30EE490A84ED060AC5
:10664000E9E600BF0AF0070101292BD0052908BFA0
:10665000677105D007291ABF00216171112121D06E
:106660002021617384ED078A174984ED088A84ED3F
:10667000098A9FED171ADFED170A4A79A27340EED7
:10668000010AC9689FED141A00222161227520EECB
:10669000011A0E4AB2FBF1F141EE000A1439C4EDC1
:1066A000060AB8E66171DBE7D651002000000CC293
:1066B000000000C3ECB20008A0030020E05100205D
:1066C000A8030020A05C00208803002040600A008E
:1066D000287EC43F00007042A69B443B00207047C8
:1066E000704770B50546007C0026002830D0402356
:1066F000022281212846FEF7BDFD4023022201210E
:106700002846FEF7B7FD0823032282212846FEF71C
:10671000B1FD4FF40770F9F715FEC5F8180200280F
:1067200008BF012612D00446D5F81C020068804735
:106730000020C4F81402C4F81802287CD4F80422FB
:10674000A8B1402301212846FEF79EFD304670BDCA
:106750004FF40073022281212846FEF78BFD4FF48F
:106760000073022201212846FEF784FDCBE74FF497
:10677000007301212846FEF787FDE7E7F8B5002101
:106780000698089CC6B2C3F30745C3F307270091D8
:10679000082E08BF002D1FD0A819082822D8394676
:1067A000234802F07BFF0121B140491EA9408DF82A
:1067B0000000C9B204FA05F28DF80110D2B2884384
:1067C0008DF80220114040EA01028DF8032039467D
:1067D000174802F09DFF25E0E2B23946144802F066
:1067E00097FF1FE005BBFEB1202E1DD8F01DC3088A
:1067F000002B12DD0DF1FF3013F0010F02D000F875
:10680000014F24125A1008D044704FEA242C00F88B
:1068100002CF4FEA2C24521EF6D16A46394604486C
:1068200002F0E8FD0020F8BD4FF0FF30F8BD000099
:10683000A05C00200020704710B501460348FEF719
:1068400069FB0248FEF746FB002010BDD00900207E
:1068500070B50546D0F8186208780C4610F0600153
:1068600025D020292BD1E288CAB110F0800F6078A2
:106870000AD0D5F81C128B6831469847E288314619
:106880002846FEF7A0FB1AE086F80002A07986F8F9
:106890000102E28831462846FEF77BFB0FE0D5F87F
:1068A0001C12607800228B682146984707E06078C8
:1068B0000A2804D1012203492846FEF784FB002060
:1068C00070BD00002002002010B580220021034886
:1068D00002F01EFF02490020086010BDA05C0020ED
:1068E0000C040020D0F81802002804BF02207047D2
:1068F0000021C0F814120846704770B50446002500
:106900008121FEF7CCFB01212046FEF7C8FB822146
:106910002046FEF7C4FBD4F8180250B1D4F81C028C
:1069200040688047D4F81802F9F73BFD0020C4F80E
:106930001802284670BD38B50446694640F2211059
:1069400000F0B4FD00281CBF4FF0FF3038BD0098A8
:106950002060002038BD70B50546D0F81842FEF71B
:106960003FFCC4F80C02D5F81802002804BF02202E
:1069700070BDD4F80402D5F81C12CA6804F503717E
:106980009047002070BD00000A2824BF4FF0FF3060
:1069900070472DE9F05FDFF8E881DDE90AC112F008
:1069A000FF0708F114094FF0000E18D0C2F3072AB0
:1069B000BAF1020F80F0DF800CF0FF05012D08BF57
:1069C000704E03D0022D14BF6F4E704E704C082DC8
:1069D00043D2DFE805F0420B0D0F1114171A08F827
:1069E00000E049F820E00020BDE8F09F694A0EE091
:1069F000694A0CE022460AE04FF2244207E047F6DB
:106A0000E01204E043F6F04201E041F6786293467A
:106A10000BEBDB7B03EB6B0B06EBD676BBEB660F6E
:106A20007CDCB2F1FF3F08BF224602EBD272741049
:106A3000A3EB62026442A24270DB584A0226584C21
:106A400012F800B0574ABBF1100F0AD0BBF1110F7A
:106A500046D0BBF1200F62D08DE04FF0FF32A3464D
:106A6000D6E7002D08BF66F3070C002908BF0821F0
:106A70000CF0FF0CBCF1030F1CBFBCF1020FBCF10A
:106A8000010F78D1022918BF042907D0082918BF9F
:106A9000102903D0202918BF40296CD108F80070B4
:106AA000BAF1000F14BF01250025255449F8203004
:106AB00082F802C001F07E00D070BCF1030F08D054
:106AC000BCF1020F08BF402907D000BF82F804E0E4
:106AD0004EE0202918BF4029F8D10120107147E06D
:106AE000002D04BF032262F3070C002908BF7E219A
:106AF0000CF0FF02032A08BF31F07E023BD108F8F8
:106B00000070BAF1000F14BF012200222254264A5D
:106B100049F8203001F07E01115429E02BE0002DCE
:106B200008BF66F3070C002908BF4FF47A410CF048
:106B3000FF0CACF10105072D1DD21C4EA1F5FA7515
:106B4000B54218D208F80070BAF1000F14BF012541
:106B50000025255449F8203082F805C0D160DDE9D0
:106B60000E0150EA010303D00C9B1370C2E904012B
:106B70000020BDE8F09F4FF0FF30BDE8F09F00001F
:106B8000CC510020E0C81000481D0E0040420F000C
:106B900048E8010020A1070090D00300ECB20008F3
:106BA000D651002088030020B00300209DCE0300B2
:106BB0000FB4022805D29DF81010012918BF022930
:106BC00003D04FF0FF3004B070470E4B9DF8042007
:106BD0001A541233029A43F8202003F108029DED63
:106BE000030A02EB800282ED000AA3F10E021154A7
:106BF0000599002918BF0121034A1154002004B04F
:106C0000704700008E030020900300200149487067
:106C1000002070478803002030B490F850104A1EBE
:106C2000102A16D2DFF858C0002200298CF8501024
:106C300023DD00BF02EB8203C45C032C09D81918C2
:106C40008D78032D05D1CD780F2D9CBF4D78032D68
:106C500003D930BC4FF0FF3070470CF80340634459
:106C60008C789C70CC78DC704C785C7009791971E8
:106C70009CF85010521C9142DCDC30BC0020704764
:106C8000B803002010B50621AC2000F07BFC0721E2
:106C9000AD2000F077FC0721AE2000F073FC172137
:106CA000A92000F06FFC5521AB2000F06BFC4221C5
:106CB000AA2000F067FC07219B2000F063FC06215E
:106CC0009C2000F05FFC0321962000F05BFC3D4C13
:106CD000607840B10321902000F054FC0421912001
:106CE00000F050FC07E00121902000F04BFC022155
:106CF000912000F047FC607840B10321CA2000F0E9
:106D000041FC0421CB2000F03DFC07E00121CA201A
:106D100000F038FC0221CB2000F034FC012180205F
:106D200000F030FC40F6FE71812000F02BFC0721C2
:106D30007F2000F027FC0121E42000F023FC01214A
:106D4000592000F01FFC0421E32000F01BFC01216E
:106D5000E52000F017FC0121E72000F013FC0221E0
:106D6000E82000F00FFC0A21EA2000F00BFCFF21D4
:106D7000EF2000F007FC8021F82000F003FC40F237
:106D8000DC51B72000F0FEFB0121C42000F0FAFB2B
:106D9000607840B10321B82000F0F4FB0421B92051
:106DA00000F0F0FB07E00121B82000F0EBFB02212E
:106DB000B92000F0E7FB0221BDE81040F12000F00F
:106DC000E1BB00008803002010B5D0E9864100290E
:106DD0001CBF94F80002FF2807D08B6894F80122AA
:106DE00021469847FF2084F80002002010BD0000D3
:106DF0004321018000487047740200204321018034
:106E00000048704730020020122008800048704778
:106E10007003002010B50A46024903A0FEF7ECF803
:106E2000004810BDBC4F002043444320436F6E66B2
:106E30006967000004200880004870476C03002048
:106E400010B50A46024903A0FEF7D6F8004810BD67
:106E5000BC4F002033454135463043324238314340
:106E60000000000010B50A46024903A0FEF7C4F86E
:106E7000004810BDBC4F002053454D5445434820A9
:106E80005069636F4757205669727475616C20436F
:106E90006F6D506F7274000043210180004870478D
:106EA000B802002010B50A46024903A0FEF7A4F874
:106EB000004810BDBC4F002043444320496E746518
:106EC00072666163650000002DE9F84FDFF80CB1D0
:106ED000B1F100090BF1100682464FF0000406F1F3
:106EE000100706F1200852DD04F1A0014FF497705D
:106EF00000F048FB012004F049F869464FF48F7018
:106F000000F0D4FA012004F041F804EB0A050098DF
:106F10000BF8050004F1A8014FF4977000F032FB64
:106F2000012004F033F869464FF48F7000F0BEFA88
:106F3000012004F02BF80098705504F1B0014FF4D3
:106F4000977000F01FFB012004F020F869464FF411
:106F50008F7000F0ABFA012004F018F80098785513
:106F600004F1B8014FF4977000F00CFB012004F01D
:106F70000DF869464FF48F7000F098FA012004F084
:106F800005F80098641C08F80500A145ACDC9BF8E6
:106F900005008BF80000737933707979397098F8AF
:106FA000052088F800208BF801007370797088F84C
:106FB00001208BF80200B370B97088F802208BF8BA
:106FC0000300F370F97088F803208BF80400337124
:106FD000397188F80420BDE8F88F000008520020BD
:106FE00010B50A46024903A0FEF706F8004810BD96
:106FF000BC4F002053544D6963726F656C656374B8
:10700000726F6E69637300000A2101800048704747
:10701000240200200FB400202DE9F04FD3B0074622
:107020009DF87CB14490BBF1020F80F02F82FE48A6
:1070300010F80B00002800F02982FC4810F80B0023
:10704000002800F023829DF87481B8F1000F1CBF66
:10705000B8F1010FB8F1020F40F018829DF87E01DF
:107060009DF886114F904B919DF884619DF87F416A
:10707000BDF88C91102803D0202823D000F006BA48
:10708000032C1CBF022C012C40F0008260980228C7
:1070900018BF042808D0082818BF102804D02028BA
:1070A00018BF402840F0F281012E18BF022E04D0F4
:1070B000032E18BF042E40F0E981B9F1FF0F00F252
:1070C000E5810EE0481EC82880F0E0816098A0F5B8
:1070D000FA71D748884240F2D981B9F1FF0F00F226
:1070E000D581DFF850A39AF85000401E10F0FF053C
:1070F00018BF9DF97D110AD005EB8500504490F929
:107100000400884203DD681E10F0FF05F4D1CA496F
:10711000AF2000F0CBF9C949B02000F0C7F9C84949
:10712000B12000F0C3F9C749B32000F0BFF905EB67
:107130008500C0494E900844BBF1000F90F803A0B1
:107140001ED0C14810F90A10BB2000F01BFABF483E
:1071500010F90A10BC2000F015FAB6494E98095CE7
:10716000C12000F00FFABA4809F1100A4FF0100CD4
:10717000017843F6095001290FD0022919D025E0E2
:10718000B44810F90A10BB2000F0FCF9B24810F91D
:107190000A10BC2000F0F6F9DFE7B0495C9A5C9B6E
:1071A000B2FBF1F24492B3FBF1F201FB123149025E
:1071B0000AE0AB495C9A5C9BB2FBF1F24492B3FBF0
:1071C000F1F201FB12310902B1FBF0F74498C3B2AE
:1071D000380A8DF800308DF801008DF80270B8F192
:1071E000010F10D19F495E988969401AA0F2DC50C6
:1071F000010E8DF80310010C8DF80410010A8DF8B2
:1072000005108DF806009DF87C11202000EA411B36
:10721000BDF88C11DDF83CE1CAB29DF88A710020FE
:10722000BDF88811BEF1100F04D0BEF1200F6ED052
:1072300000F02CB905F00F054BEA05058DF8075055
:10724000609D8DF80800102D08BF0A2515D00CDCB4
:10725000022D08BF072510D0042D08BF08250CD02B
:10726000082D08BF092508D009E0202D08BF0B25EF
:1072700003D0402D08BF0C2501D18DF80950012EF7
:1072800004BF9DF8095045F0100514D0022E04BF2C
:107290009DF8095045F020050DD0032E04BF9DF840
:1072A000095045F0300506D0042E04BF9DF8095062
:1072B00045F0400501D18DF809502FB99DF80950CE
:1072C00045F080058DF809508DF80A20012C08BF83
:1072D000022208D0022C08BF012204D0032C08BFD0
:1072E0008DF80B0001E08DF80B209DF88B21012A11
:1072F00005D19DF80B2042F004028DF80B20032CE1
:1073000006D0022C04BF609A402A06D00BE039E078
:10731000609A202A18BF402A05D19DF80B2042F020
:1073200008028DF80B209DF88521012A05D19DF8D2
:107330000B2042F010028DF80B20002908BF062117
:1073400003D0042938BF042101D2ADF8881189B2D5
:107350000A0A8DF80C208DF80D108DF80E008DF8AE
:107360000F0003F03F008DF80000012C08BF40F033
:10737000800004D0032C08BF40F040003DD18DF8C0
:1073800000003AE005F00F0C8DF808004BEA0C0CF9
:107390004B984CF0100C8DF809008DF807C08DF853
:1073A0000A20002F14BF0020022040F009008DF8B1
:1073B0000B00002908BF052003D0032938BF032094
:1073C00001D2ADF88801BDF888018DF81020010ABE
:1073D0008DF80C108DF80D00234960984FF0110CBA
:1073E000B1FBF0F0010A8DF80E108DF80F0003F0DC
:1073F0007F008DF800000AF1010A0DEB0C004A46EF
:107400000DF5C771F9F797FB002140F2451000F028
:10741000B9F80021052000F0B5F81FFA8AF2694694
:107420000620FEF729FF21E0900300208E030020B4
:107430009DCE0300B8030020BC510020C0510020A5
:10744000C4510020C851002028520020385200208A
:1074500092030020085200201852002080841E0051
:1074600000093D00A05C00200048E801B8F1000FD1
:1074700004BF0121B42010D0B8F1010F04BF0121D5
:10748000B5200AD0B8F1020F0AD000BF4FF0FF308C
:1074900053B0BDE8F00F5DF814FB00F073F803E0A3
:1074A0000121B62000F06EF80020F1E72DE9F84345
:1074B0000F46314900EB400001EB8000D0E9004568
:1074C00060B2B0F1FF3F07D02C4804F00302002166
:1074D00002602B4802F01CF900200646C4F307485E
:1074E000EDB2009008EB050008281BD8C4F3072173
:1074F000234802F0D3F8C5F108018DF80000A1EB94
:1075000008029040C0B2220E8DF80100012A12BF7D
:10751000C8409DF9010008418DF8020018BFC0B2B3
:1075200038601EE0B8F1000F1BD1D5B1202D18D85E
:10753000E81D4FEAD008C4F3072143466A461048C5
:1075400001F09AFEB8F1010058BF694604D40A5C04
:10755000401E02EB0626FAD5200E012818BF3E6019
:1075600002D00020BDE8F883C5F1200006FA00F142
:1075700041FA00F03860F4E704B300080C0400207E
:10758000A05C0020B0F5A37F24BF4FF0FF30704710
:10759000F0B50C461B4983B010B1012808D00AE0B1
:1075A00004F003020A600021174802F0B1F826E057
:1075B00014F0010F23D1154A00EB400002EB8000CC
:1075C000D0E900568768C6F30720012802BF4FF0B4
:1075D000FF3003B0F0BD68B2B0F1FF3F06D005F058
:1075E00003020A600021084802F092F80096002287
:1075F000CDE901742B4611461046FFF7BFF803B0E2
:107600000020F0BD0C040020A05C002004B30008A2
:107610002DE9F84F012631461220FFF7B3FF012173
:107620001320FFF7AFFFF74C04F1080001F06DFCE9
:10763000E169401AA0611F214D20FFF7A3FF00213F
:107640004C20FFF79FFFF04CAF202168FFF79AFF17
:10765000B0206168FFF796FFB120A168FFF792FFA5
:10766000B320E168FFF78EFFFFF70CFBE74C2068C3
:10767000002800F09882E64D7103B0FBF5F0B1FBF5
:10768000F0F000EE100AB8EE400ABCEEC00A10EEB0
:10769000101A3F2988BF3F218C20FFF773FF206815
:1076A0004FF40041B0FBF5F0B1FBF0F000EE100A32
:1076B000B8EE400ABCEEC00A10EE101A3F2988BF8F
:1076C0003F21D220FFF75EFFD24D4FF00108691E27
:1076D000287801280CBF40460020012291F802C002
:1076E0000023032411F10101BCF1000F11F8027F06
:1076F00018BF08FA02FC604491F801C0C0B2002F24
:107700001CBF571C08FA07F73B44921CDBB2641EEF
:10771000EAD1E9791844C0B2012914BF00218021BF
:107720000844DFF8F4A2C7B243F60959DAF80000BA
:10773000400190FBF9F15C20FFF724FFDAF8040028
:10774000400190FBF9F15D20FFF71CFFDAF808001B
:10775000400190FBF9F15E20FFF714FFDAF80C000E
:10776000400190FBF9F15F20FFF70CFFDAF8100001
:10777000400190FBF9F16020FFF704FFDAF81400F4
:10778000400190FBF9F16120FFF7FCFEDAF81800E8
:10779000400190FBF9F16220FFF7F4FEDAF81C00DB
:1077A000400190FBF9F16320FFF7ECFEAAF114040D
:1077B000DFF86882207801280CBF98F800100021BB
:1077C0006820FFF7DFFE607801280CBF98F80110F1
:1077D00000216920FFF7D6FEA07801280CBF98F899
:1077E000021000216A20FFF7CDFEE07801280CBFCF
:1077F00098F8031000216B20FFF7C4FE20790128C0
:107800000CBF98F8041000216C20FFF7BBFE6079D4
:1078100001280CBF98F8051000216D20FFF7B2FE7B
:10782000A07901280CBF98F8061000216E20FFF700
:10783000A9FEE07901280CBF98F8071000216F20FD
:10784000FFF7A0FE60219720FFF79CFE012110208A
:10785000FFF798FEDAF82000400190FBF9F1642070
:10786000FFF790FE207ADFF8B88101287ED0002152
:107870000F20FFF787FE00BFDAF82400400190FBDD
:10788000F9F16520FFF77EFE98F80000411EE62022
:10789000FFF778FE98F80000411EF420FFF772FE13
:1078A00098F80000C0F10800C200D8E90401F8F718
:1078B0009FFD89460146ED20FFF764FE4946EE2014
:1078C000FFF760FE607A01287DD000211120FFF7CC
:1078D00059FEA0200121FFF755FEA2200021FFF74D
:1078E00051FE00210920FFF74DFEA2200121FFF7E4
:1078F00049FEA1200121FFF745FEA3200021FFF74B
:1079000041FE00210920FFF73DFEA3200121FFF7E2
:1079100039FE0121A020FFF735FE0121A120FFF74C
:1079200031FE00219D20FFF72DFE00219E20FFF754
:1079300029FE00219F20FFF725FE00215B20FFF795
:1079400021FE0021A020FFF71DFE0021A120FFF74E
:1079500019FE20214FF49770FFF714FE69464FF48B
:107960008F70FFF7A3FD0098C0B200E003E0042889
:1079700040F019817AE0297AD920FFF703FE98F8C0
:10798000020001280ED0022807D0032840F00B8106
:107990000021D820FFF7F6FD08E00121D820FFF7ED
:1079A000F1FD03E00221D820FFF7ECFD98F8030079
:1079B00010281DD008DC02280BD004280ED008287F
:1079C00011D000F0F0B83BE0202816D0402829D094
:1079D000E9E00721DE20FFF7D5FD27E00821DE20C2
:1079E000FFF7D0FD22E00921DE20FFF7CBFD1DE0EF
:1079F0000A21DE20FFF7C6FD18E00B21DE20FFF78D
:107A0000C1FD13E0A05C0020BC510020A0030020B9
:107A100040420F00D6510020E0510020B00300206A
:107A2000880300200C21DE20FFF7ACFD98F804103D
:107A3000DD20FFF7A7FD01210F20FFF7A3FD1BE7C6
:107A4000697AEB20FFF79EFD5D49D8F80C00B1FB89
:107A5000F0F1EC20FFF796FD98F80510E220FFF713
:107A600091FD01211120FFF78DFD32E7202140F229
:107A70002D10FFF787FD694640F21D10FFF716FD38
:107A80000098C0B201287DD1642003F08DFA6946C8
:107A90005020FFF70BFD0098102873D1494C0025AA
:107AA00094F85000002825DD10215B20FFF76AFDC7
:107AB000304603F079FA05EB85002044817842785E
:107AC0000901C07801EB82110844C1B25B20FFF7C5
:107AD00059FD304603F068FA69465020FFF7E6FC8E
:107AE000009905F1300081425DD194F850006D1C81
:107AF000A842D9DCC0B2102814D210215B20FFF7B5
:107B000041FD304603F050FA11215B20FFF73AFDAA
:107B1000304603F049FA69465020FFF7C7FC009849
:107B2000302840D110215B20FFF72CFD304603F0B8
:107B30003BFA03215B20FFF725FD304603F034FAC2
:107B400069465020FFF7B2FC009833282BD1102152
:107B50005B20FFF717FD304603F026FA00215B207B
:107B6000FFF710FD304603F01FFA69465020FFF77B
:107B70009DFC0098302816D110215B20FFF702FDF4
:107B8000304600E00FE003F00FFA39465B20FFF7C4
:107B9000F9FC304603F008FA69465020FFF786FCEE
:107BA0000098402803D04FF0FF30BDE8F88F002147
:107BB0004FF49E70FFF7E6FC0020BDE8F88F000050
:107BC0000048E801B803002070B504464FF417716F
:107BD000F9F728F80021C4F85C12C4F86012C4F860
:107BE0006412C4F86812C4F86C12C4F87012C4F8B5
:107BF0007412C4F87812C4F87C12C4F88012C4F865
:107C00008412C4F88812C4F88C12C4F89012C4F814
:107C10009412C4F898120125C4F87459C4F8601974
:107C2000D4F8780904F516620128D4F880090168AF
:107C30004B6813D004F517719847C4F8745900BF06
:107C4000D4F874090028FBD1C4F8745904F52770DE
:107C5000BDE8704040F2C461F8F7E4BF21469847A0
:107C6000F4E7000010B5044690F89E0294F89D12C7
:107C7000042202EB0121084482B2D4F88009016891
:107C80008B6804F52771984794F87C09012818BF80
:107C900010BDC82003F07AF9BFF34F8F0548016883
:107CA000054A01F4E06111430160BFF34F8F00BF4B
:107CB000FDE700000CED00E00400FA0510B5D0F877
:107CC0008009016809688847BDE810404FF47A7060
:107CD00003F05CB9A1F161001A2810D2DFE800F0CE
:107CE0000D0D0D0D0F0D0F0D0D0D0F0D0D0D0F0DBC
:107CF0000D0D0D0D0D0F0D0D0D0D01207047002008
:107D0000704700002DE9F047044600202178ADF5CA
:107D1000AD6D002909BF00208DF810110DF5AD6D76
:107D2000BDE8F08761391A2930D2DFE801F00D0D86
:107D30000D0D2F0D2F0D0D0D2F0D0D0D2F0D0D0DEB
:107D40000D0D0D2F0D0D0D0D9DF8101161391A2916
:107D500080F0E485DFE811F0CF021703A6031204D8
:107D6000E2055004E205E00320054205E205520564
:107D7000C005D005E2055B01FA0428006F00BE00D3
:107D80000D01E205A901F2013B02870200206B21EF
:107D900084F89C1284F89D0284F89E0284F89F0265
:107DA0000DF5AD6DBDE8F08760788DF81101A37811
:107DB0004FF0FF368DF8123106EB0020E1781D18E8
:107DC000002D19DDE01C0DF2131213F0010F04D188
:107DD00010F8013F8DF81431521C90F801C06B105F
:107DE0000AD000BF10F8025F82F801C090F801C00D
:107DF00002F8025F5B1EF5D19DF811219DF812017A
:107E000006EB0222801804D4221844AB18441279DD
:107E10000271FE4801F042FC722184F89C1200219C
:107E200084F89D12012184F89E1284F89F1284F830
:107E3000A00200F07EB960788DF81101A3784FF0B0
:107E4000FF368DF8123106EB0020E1781D18002D69
:107E500018DDE01C0DF2131213F0010F04D110F81D
:107E6000013F8DF81431521C90F801C06B1009D0FD
:107E700010F8025F82F801C090F801C002F8025FBA
:107E80005B1EF5D19DF811219DF8120106EB02222F
:107E9000801804D4221844AB1844127902719DF85A
:107EA00015019DF8142100EB0223732084F89C0235
:107EB0009DF8140184F89D029DF8150184F89E0236
:107EC000012084F89F0204F52872D04801F044FA9A
:107ED00000F02FB960788DF81101A3784FF0FF36CC
:107EE0008DF8123106EB0020E1781D18002D19DD08
:107EF000E21C0DF2131013F0010F04D112F8013F30
:107F00008DF81431401C92F801C06B100AD000BFEC
:107F100012F8025F80F801C092F801C000F8025F19
:107F20005B1EF5D19DF811219DF8120106EB02228E
:107F3000801804D4221844AB1844127902719DF8B9
:107F400015019DF8142100EB0223742084F89C0293
:107F50009DF8140184F89D029DF8150184F89E0295
:107F6000012084F89F0204F52872A84801F02AFA3B
:107F7000DFE060788DF81101A3784FF0FF368DF8BF
:107F8000123106EB0020E1781D18002D18DDE01CF1
:107F90000DF2131213F0010F04D110F8013F8DF808
:107FA0001431521C90F801C06B1009D010F8025F18
:107FB00082F801C090F801C002F8025F5B1EF5D1A3
:107FC0009DF811219DF8120106EB0222801804D4BD
:107FD000221844AB1844127902719DF815019DF8DE
:107FE000142100EB0223752084F89C029DF81401F3
:107FF00084F89D029DF8150184F89E02012084F802
:108000009F0204F52872814801F07CF991E06078C4
:108010008DF81101A3784FF0FF368DF8123106EB81
:108020000020E1781D18002D18DDE01C0DF2131260
:1080300013F0010F04D110F8013F8DF81431521CD8
:1080400090F801C06B1009D010F8025F82F801C0EF
:1080500090F801C002F8025F5B1EF5D19DF8112176
:108060009DF8120106EB0222801804D4221844ABBA
:108070001844127902719DF815019DF8142100EB46
:108080000223702084F89C029DF8140184F89D025C
:108090009DF8150184F89E02012084F89F0204F5E2
:1080A00028725A4801F0E8F843E060788DF8110131
:1080B000A3784FF0FF368DF8123106EB0020E178FF
:1080C0001D18002D18DDE01C0DF2131213F0010F26
:1080D00004D110F8013F8DF81431521C90F801C002
:1080E0006B1009D010F8025F82F801C090F801C04F
:1080F00002F8025F5B1EF5D19DF811219DF8120177
:1081000006EB0222801804D4221844AB18441279DA
:1081100002719DF814213D4801F0FAFA772084F8A5
:108120009C02002084F89D0284F89E02012084F8BD
:108130009F020DF5AD6D0120BDE8F08760788DF8E8
:10814000110194F802C04FF0FF370CEB00238DF8BB
:1081500012C107EB0020E1780CEB0006002E18DDC1
:10816000E01C0DF213121CF0010F04D110F801CF26
:108170008DF814C1521C45785FEA660C09D000BF27
:1081800010F8026F5570457802F8026FBCF1010CCF
:10819000F6D19DF811219DF8120107EB02228018FB
:1081A00005D422180DF5887C60441279027145AA25
:1081B000164801F08DF9782084F89C02002084F89C
:1081C0009D0284F89E02012084F89F02B1E7607846
:1081D0008DF8110194F802C04FF0FF370CEB00232B
:1081E0008DF812C107EB0020E1780CEB0006002EA1
:1081F0001BDDE01C0DF213121CF0010F04D110F86E
:1082000001CF8DF814C1521C457801E0A05C00201C
:108210005FEA660C09D000BF10F8026F5570457810
:1082200002F8026FBCF1010CF6D19DF811219DF806
:10823000120107EB0222801805D422180DF5887C64
:1082400060441279027145AAFE4801F075F979205F
:1082500084F89C02002084F89D0284F89E0201208C
:1082600084F89F0265E760788DF8110194F802C0E8
:108270004FF0FF370CEB00238DF812C107EB002005
:10828000E1780CEB0006002E17DDE01C0DF2131256
:108290001CF0010F04D110F801CF8DF814C1521C4D
:1082A00045785FEA660C08D010F8026F5570457883
:1082B00002F8026FBCF1010CF6D19DF811219DF876
:1082C000120107EB0222801805D422180DF5887CD4
:1082D00060441279027145AADA4801F0D1F87A2097
:1082E00084F89C02002084F89D0284F89E020120FC
:1082F00084F89F021DE760788DF8110194F802C0A0
:108300004FF0FF370CEB00238DF812C107EB002074
:10831000E1780CEB0006002E17DDE01C0DF21312C5
:108320001CF0010F04D110F801CF8DF814C1521CBC
:1083300045785FEA660C08D010F8026F55704578F2
:1083400002F8026FBCF1010CF6D19DF811219DF8E5
:10835000120107EB0222801805D422180DF5887C43
:1083600060441279027145AAB64801F043F86120D1
:1083700084F89C02002084F89D0284F89E0201206B
:1083800084F89F02D5E6607800268DF81101A27866
:10839000771E07EB002002EB000C4FF49679354670
:1083A0008DF81221BCF1000F16DDE01C0DF2131147
:1083B00012F0010F04D110F8012F8DF81421491C7F
:1083C00043785FEA6C0207D010F802CF4B70437815
:1083D00001F802CF521EF7D19DF811119DF812013C
:1083E00007EB0121401804D4211844AA104409794C
:1083F00001719DF814019449FDF792FFB0F1000C52
:108400004FF0620084F89C024FF0010101EBEC7028
:1084100084F89F0284F8A0C24FF00007C4BFDFF8C1
:108420002882A9F5807236DDC7EB071000EB8000CB
:1084300008EB8001488D8318002B28DD0023504075
:1084400010F0010005D005EB04090B7889F8A13282
:108450000123B1F82A909144814515DD05EB030A0B
:1084600011F80390A2445B1C8AF8A19205EB030A61
:10847000A24411F803908AF8A192B1F82A90801CC6
:1084800091445B1C8145E9DC488D304486187F1C93
:108490003546BC45C8DC701C010A84F89D1284F87E
:1084A0009E0246E660788DF81101A2788DF81221BF
:1084B00094F803C012EB002019D0E01C0DF28F31AC
:1084C00012F0010F03D010F8012F01F8012F9DF8D1
:1084D00012219DF8113102EB0322520807D0437894
:1084E0004B7010F8023F01F8023F521EF7D1DDE950
:1084F000E701CDE90001DDE9E4126046E69BFEF705
:1085000057FB632184F89C12002184F89D1284F8A3
:108510009E1200286FD017E160788DF81101A278C3
:108520008DF8122112EB002019D0E01C0DF2C7418A
:1085300012F0010F03D010F8012F01F8012F9DF860
:1085400012219DF8113102EB0322520807D0437823
:108550004B7010F8023F01F8023F521EF7D10DF5A3
:108560009960FEF759FB682184F89C12002184F879
:108570009D1284F89E1200283DD0E5E060788DF8C9
:108580001101A2788DF8122194F803C012EB00209B
:1085900019D0E01C0DF26F3112F0010F03D010F86A
:1085A000012F01F8012F9DF812219DF8113102EBE6
:1085B0000322520807D043784B7010F8023F01F8AD
:1085C000023F521EF7D1DEAF97E86F008DE86F00D3
:1085D000DDE9DC236046FEF7D7F9642184F89C12BC
:1085E000002184F89D1284F89E12002803D0ABE08D
:1085F00084F89F029DE5A5E00DF5AA6000F09BFCC4
:1086000060788DF81101A2788DF8122112EB00200C
:108610001ED0E01C0DF2A73112F0010F03D010F8AC
:10862000012F01F8012F9DF812219DF8113102EB65
:10863000032252080CD043784B7010F8023F01F827
:10864000023F03E0A05C00208C5D0020521EF2D1AE
:10865000B94DB5F90000B0F1FF3F04D13422B7A104
:10866000C6A001F0E9FEA888E96800040860C94DC9
:1086700001266E712E714FF48872EEA96846F8F7E4
:108680009FFAEAAF97E80F00FEF7C4FC0DF5AC6166
:10869000BD20FEF70BFFDDF8600501281BD00DF5AE
:1086A000AA6000F014FC0DF5AA6000F01EFCBA4EA2
:1086B000287938B10DF5AA6000F0D0FB10EE100A51
:1086C000B042F5DB0DF5AA6000F0E8FB95F820005C
:1086D00001281BD10AE0662084F89C02002084F85F
:1086E0009D0284F89E0284F89F6222E50DF24C50B0
:1086F000FEF721F905F1080000F007FCDDF84C1544
:10870000401A3C30E861002085F82000A14801F0C3
:108710003DF8894DB5F90000B0F1FF3F04D1342296
:1087200086A196A001F088FEE96868680860FEF7F7
:108730006FFF662184F89C12002184F89D1284F852
:108740009E1208B9012053E7002051E7DBA8FEF78D
:10875000F2F801008F48DB9A806910444FF07102F3
:10876000DB9084F89C224FF0000284F89D224FF0A9
:10877000040284F89E220CBF0121002184F89F127C
:10878000010E84F8A012010C84F8A112010A84F8E9
:10879000A21284F8A302CCE461788DF81111A278BA
:1087A0008DF8122102EB0122002AC8BF0DF264539A
:1087B00005DD211809791954401C8242F9DCDDF8E5
:1087C0006405FEF723FA692184F89C12002184F8DD
:1087D0009D1284F89E120028B6D1B3E76179207902
:1087E000FEF772FB6A2084F89C02002084F89D0248
:1087F00084F89E02012084F89F029AE460788DF844
:108800001101A2784FF0FF3505EB002C02EB0C00B4
:108810008DF81221002817DDE01C0DF2131112F063
:10882000010F04D110F8013F8DF81431491C437831
:108830006244521008D000BF10F802CF4B7043784A
:1088400001F802CF521EF7D19DF811119DF81201C7
:1088500005EB0121401804D4211844AA10440979D9
:108860000171E0792179A27900EB01606179090455
:1088700001EB022101446C2084F89C02002084F862
:108880009D02082284F89E22A1F18572921F08BFE2
:10889000012084F89F024148007884F8A0024048F3
:1088A000007884F8A1023F48007884F8A2023E488C
:1088B000007884F8A3023D48007884F8A4023C487C
:1088C000007884F8A5023B48007884F8A6023A486C
:1088D000007884F8A7022CE4FDF7F6FF6D2084F8F9
:1088E0009C02002084F89D0284F89E02012084F8F6
:1088F0009F0284F87C091CE410213048FDF778FCC5
:108900006E2084F89C02002084F89D0284F89E0268
:10891000012084F89F0284F87C090AE46B2084F823
:108920009C02002084F89D0284F89E0284F89F0235
:108930000DF5AD6DBDE8F0877C5D00206D6265646E
:108940002D6465762F746172676574732F68616C2E
:108950002F5441524745545F53544D2F5441524771
:1089600045545F53544D333246342F6770696F5FFF
:108970006F626A6563742E68000000006F626A2D82
:108980003E70696E20213D202850696E4E616D65F4
:10899000294E4300A05C002000002041187AFF1FF0
:1089A000197AFF1F1A7AFF1F1B7AFF1F107AFF1F09
:1089B000117AFF1F127AFF1F137AFF1F00100108A0
:1089C00070B50025044680F87C59042000F076FF3D
:1089D00008B104490160C4F87859C4F880092046F8
:1089E00070BD00005CC3000870B504460068416AB1
:1089F00020468847206801220021036920469847C5
:108A00000546B0F1FF3F206811D002220369002122
:108A100020469847064620680022294603692046DA
:108A200098472068816A20468847304670BD816A31
:108A3000204688474FF0FF3070BD704770470000F8
:108A400070B50546174C164828602068002804BFFA
:108A5000201D2060261DB04204D056221249134822
:108A600001F0EAFC00211248D4F8003010228C46B4
:108A700050F82140AC4208BF40F821C0491C521EAA
:108A8000F6D10849002B12BF0868081D0860B042E3
:108A900004D056220449054801F0CEFC284670BD9A
:108AA0007CC300080C0200200CC50008F8C40008B4
:108AB0009009002010B50C46483002F039F82046E5
:108AC00010BD00EB011000F19401D0F8A020002AA5
:108AD00008BF70478868104770B50446483001F0F9
:108AE00079FF236C054600F47C52002B18BF002A46
:108AF00003D004F13401E06B9847236B05F0FC02CE
:108B0000002B14BF002A70BD04F12401E06ABDE807
:108B10007040184770B50E46044620491E48154659
:108B20002060D1E902230021A260E3601C4A226197
:108B3000A161646104F10801E1611A492162BFF396
:108B40006F8FBFF34F8F00216162216361632164E6
:108B500084F8441084F845104C2104F14800F8F7DB
:108B600061F802231022104904F1940000F0F2FE93
:108B7000A0F194044FF41650C4F8B4002A463146CC
:108B800004F1480001F042FE2246084904F1480081
:108B900001F014FF204670BDB0C30008DCB200082D
:108BA0009FE8078059B000083D2C0008C38A0008E0
:108BB000002908BF704701290AD0022918BF704751
:108BC00000F13401026C002A08BF70478868104722
:108BD000026B00F12401002AF8D1704770B50D46F0
:108BE000044601F08BF8E868002804F134000DD049
:108BF000A9688160D5E90012C0E90012E968C16086
:108C000001220221203801F0FBFA08E00021016076
:108C1000C1600A46022104F1140001F0F1FABDE836
:108C2000704001F0BFB8000070B504460D48002246
:108C3000C4E90002A260E26022616261A261E261B5
:108C4000226262622263626322640D462346064A00
:108C500004F1140001F032FA2946201D01F05DF9FB
:108C6000204670BDC8C30008B18B000810B504468B
:108C70000348206004F1140001F0FAF9204610BD09
:108C8000C8C300080021F7F7A5BE00000748016827
:108C9000002904BF011D0160001D814208BF70470B
:108CA00056220349034801F0C7BB00001802002008
:108CB0000CC50008F8C4000870B5044600680E46EC
:108CC00041682046884720684168204688470F4D04
:108CD0002868A0420AD0D4E90A120023201D01F01E
:108CE00039FF201D216B01F069FF2C60206881682D
:108CF000204688473146201D02F086F80546206848
:108D0000816820468847284670BD00001402002074
:108D100070B5044600680D461646416820468847EF
:108D2000C4E90A560F4D002028602068416820469B
:108D300088472868A0420AD0D4E90A120023201DDF
:108D400001F008FF201D216B01F038FF2C60206826
:108D5000816820468847206881682046BDE87040C9
:108D6000084700001402002007480168002904BFDA
:108D7000011D0160001D814208BF70475622034952
:108D8000034801F059BB0000180200200CC5000880
:108D9000F8C4000870B5044600680D4641682046D6
:108DA000884725630F4D00202860206841682046D1
:108DB00088472868A0420AD0D4E90A120023201D5F
:108DC00001F0C8FE201D216B01F0F8FE2C60206828
:108DD000816820468847206881682046BDE8704049
:108DE000084700001402002038B504461848DDF892
:108DF00010C0206000206060A060E06020616061C1
:108E0000A061E06108252062C4E90905E06211481B
:108E10002063201DCDF800C001F02CFF20684168C0
:108E2000204688470C4D2868A0420AD0D4E90A128F
:108E30000023201D01F08EFE201D216B01F0BEFEDF
:108E40002C602068816820468847204638BD000095
:108E5000D8C3000840420F001402002070B5044639
:108E600000F04CFF00F04AFF2068002520B1E068C8
:108E700002F009F86168451A00F094FFA0682C1808
:108E800000F090FF00EE104A9FED031AF8EEC00AC2
:108E900080EE810A70BD00000024744970B504465C
:108EA00000F02CFF00F02AFF2068002520B1E068C8
:108EB00001F0E9FF6168451A00F074FFA0682844DA
:108EC000A06000202060BDE8704000F06BBF10B5CE
:108ED000044600F013FFE06801F0D5FF6060002059
:108EE000A060BDE8104000F05DBF10B5044600F082
:108EF00005FF206828B9E06801F0C5FF6060012027
:108F00002060BDE8104000F04DBF70B5044600F091
:108F1000F5FE00F0F3FE2068002520B1E06801F0C6
:108F2000B2FF6168451A00F03DFFA0682C1800F000
:108F300039FF204670BD70B50025056045600446C8
:108F4000856000F083FFE06000F0D8FEE06801F08B
:108F50009AFFC4E9010500F025FF204670BD00001E
:108F600010B51C46FFF7D6FD2146B83000F046F894
:108F7000044940F8B81D5C31C0F8BC103C39C0F859
:108F8000B81010BDF4C3000810B5074940F8BC1B69
:108F90005C3140F804193C39016000F04FF8034996
:108FA00040F8B81D10BD0000F4C30008B0C30008AD
:108FB0000020704700207047002070472DE9F041E5
:108FC000054600680F460C468E18416A28468847B9
:108FD000B4420AD0286814F8011BC26A2846904798
:108FE000B0F1FF3F18BFB442F4D12868816A284627
:108FF0008847E01BBDE8F0810020704710B584B0C1
:1090000000F0A8F804460A4820603C306060002068
:109010006061224607A16846F7F710FA06A1684684
:10902000F7F7B1FC6061FFF72DFE04B0204610BDDC
:1090300060C400083A257000772B000010B5044684
:10904000054820603C3060606069F7F7CDFC204641
:10905000BDE8104000F090B860C40008007B704785
:1090600070B506460D46154801F0D6FF1448046851
:10907000F4B1A068C8B12A463146F7F711FDA0B98E
:10908000A068F7F7EEFCA8420FD10C480168002950
:1090900004BF011D0160001D814204D05622094910
:1090A000094801F0C9F9204670BD6468002CE0D180
:1090B000024801F0B1FF002070BD0000F401002063
:1090C000F00100200CC50008F8C4000870B5044683
:1090D0000B480026A160C4E900060D46227309482A
:1090E00001F09AFF002D08BF666003D006480168B2
:1090F00061600460034801F08FFF204670BD0000EE
:10910000ACC40008F4010020F001002010B50446B2
:109110000D4820600D4801F07FFFA06878B10C4930
:109120000868A04204BF6068086008D04168A14296
:1091300003D008464968A142FBD1616841600348F9
:1091400001F06AFF204610BDACC40008F401002005
:10915000F001002010B5064A40F8042B0022FFF76A
:10916000B5FF044940F8041D3431416010BD0000D2
:109170007CC30008BCC4000810B5001DFFF7C6FF83
:10918000BDE81040001FFFF75BBC10B50446406807
:1091900028B1FFF763FF012804BF606810BD0020FD
:1091A00010BD10B50446406810B1FFF757FF08B175
:1091B000002010BD6068002818BF001F10BD406867
:1091C000002818BF0120704710B54068002808BF6C
:1091D00010BDFFF743FF00280CBF0120002010BD89
:1091E0000068704710B50446002020606060087871
:1091F0002F280DD1487858B14B1C002123602268DC
:1092000010782F2806D038B1501C491C2060F6E792
:10921000204610BD501C20601846FFF721FF6060FB
:10922000204610BD084882B0016841F0800101600D
:109230000648016841F480410160006800F4804004
:10924000009002B0FBF782BA343802404438024042
:1092500008461146F9F7F8BC70B514460D4612F0F1
:109260003F0F04BF501C84B221462846F9F7F8FC92
:109270000028F9D170BD00002DE9F0471E461746C1
:10928000894604464FF0000872B600F12405B0F993
:109290002400B0F1FF3F05D11949342201F140000B
:1092A00001F0CAF8A888E968000408600A2001F003
:1092B0007BFE09F07F0104F14400FFF7FDFC00256F
:1092C000002E08DD002104F14400FFF7F5FC78557D
:1092D0006D1CAE42F6DC012001F066FE34F9240F6D
:1092E000B0F1FF3F05D10649342201F1400001F001
:1092F000A3F8E1686068086062B64046BDE8F087A0
:10930000DC9700082DE9F0411E1E174604464FF079
:10931000000872B6454608DD002104F14400FFF75D
:10932000CBFC78556D1CAE42F6DC012001F03CFE12
:1093300034F9240FB0F1FF3F05D10649342201F181
:10934000400001F079F8E1686068086062B6404664
:10935000BDE8F081DC9700082DE9F0471E4617466E
:10936000894604464FF0000872B600F12405B0F9B2
:109370002400B0F1FF3F05D11149342201F1400032
:1093800001F05AF8A888E96800040860012001F09B
:109390000BFE09F07F0104F14400FFF78DFC00256E
:1093A000002E08DD002104F14400FFF785FC78550C
:1093B0006D1CAE42F6DC62B64046BDE8F0870000A8
:1093C000DC9700082DE9F0411D1E164607464FF0B8
:1093D000000872B6444608DD002107F14400FFF79B
:1093E0006BFC3055641CA542F6DC62B64046BDE815
:1093F000F08100002DE9F0471F469046894604465B
:10940000002572B600F12406B0F92400B0F1FF3F48
:1094100005D11A49342201F1400001F00DF8B0885D
:10942000F16800040860012001F0BEFD09F07F0032
:1094300040F0800104F14400FFF73EFC002F08DDFE
:1094400018F8051004F14400FFF736FC6D1CAF421C
:10945000F6DC012001F0A8FD34F9240FB0F1FF3F44
:1094600005D10649342201F1400000F0E5FFE16832
:109470006068086062B6BDE8F0870000DC9700080D
:109480002DE9F0411E1E174604464FF0000572B646
:1094900007DD795D04F14400FFF70EFC6D1CAE4260
:1094A000F7DC012001F080FD34F9240FB0F1FF3F1B
:1094B00005D10649342201F1400000F0BDFFE1680A
:1094C0006068086062B6BDE8F0810000DC970008C3
:1094D0002DE9F0471F46904689460446002572B69E
:1094E00000F12406B0F92400B0F1FF3F05D1114985
:1094F000342201F1400000F09FFFB088F1680004C1
:109500000860012001F050FD09F07F0040F080016B
:1095100004F14400FFF7D0FB002F08DD18F8051018
:1095200004F14400FFF7C8FB6D1CAF42F6DC62B6E5
:10953000BDE8F087DC9700082DE9F0411D1E1646B6
:1095400007464FF0000472B607DD315D07F14400B5
:10955000FFF7B2FB641CA542F7DC62B6BDE8F08100
:10956000F0B5444D044685B0B5F90000B0F1FF3FB9
:1095700005D14149342201F1400000F05DFFE96866
:10958000686808603D4DB5F90000B0F1FF3F05D1B6
:109590003949342201F1400000F04EFFE968686863
:1095A0000860B4F9340004F13405B0F1FF3F05D18F
:1095B0003149342201F1400000F03EFFE96868685B
:1095C00008600A2001F0F0FCB4F9340004F134051D
:1095D000B0F1FF3F05D12849342201F1400000F0ED
:1095E0002BFFA888E968000408600A2001F0DCFC71
:1095F000B4F9240004F12405B0F1FF3F05D11E4960
:10960000342201F1400000F017FFE9686868086043
:109610000A2001F0BBFC0022082104F14400FFF7FE
:1096200077FB174904F14400FFF7B4FB154804F138
:109630007807D0E9005600F061FB1348CDE90056E9
:10964000CDE9024069463846FFF7C8FA00F0AAFBA8
:10965000012084F8200000206071A06104F108005E
:10966000FFF735FC04F10800FFF73FFC05B00120CF
:10967000F0BD00005C5D0020DC9700087C5D0020F0
:1096800000127A004CC2000845B0000872B6417959
:10969000012904BF0021017162B6704770B50E4602
:1096A000044672B600F12405B0F92400B0F1FF3F82
:1096B00005D11649342201F1400000F0BDFEA88812
:1096C000E96800040860012001F06EFC06F07F01EB
:1096D00004F14400FFF7F0FA002104F14400FFF721
:1096E000EBFAC5B2012001F05FFC34F9240FB0F1B0
:1096F000FF3F05D10549342201F1400000F09CFEF6
:10970000E1686068086062B6284670BDDC970008B2
:109710002DE9F04117460E46044672B600F12405C5
:10972000B0F92400B0F1FF3F05D11749342201F10F
:10973000400000F081FEA888E9680004086001206C
:1097400001F032FC06F07F0040F0800104F144009B
:10975000FFF7B2FA394604F14400FFF7ADFA0120F1
:1097600001F022FC34F9240FB0F1FF3F05D1064986
:10977000342201F1400000F05FFEE168606808609B
:1097800062B6BDE8F0810000DC97000870B50446C1
:1097900000F13405B0F93400B0F1FF3F04D13422B8
:1097A0000EA11EA000F048FEE968686808600A2063
:1097B00001F0FAFB34F9340FB0F1FF3F04D1342249
:1097C00006A116A000F038FEA088E1680004086039
:1097D000BDE870400A2001F0E7BB00006D626564DF
:1097E0002D6465762F746172676574732F68616C80
:1097F0002F5441524745545F53544D2F54415247C3
:1098000045545F53544D333246342F6770696F5F50
:109810006F626A6563742E68000000006F626A2DD3
:109820003E70696E20213D202850696E4E616D6545
:10983000294E43002DE9F84F0E46DDE90A5A164934
:10984000DDF830B09846914640F8081BFFF773FBEF
:10985000A0F10804002740F81C7F3146476087606C
:10986000C76000F06FFB6763A763E76304F1340030
:109870005946276400F066FB781E00902B4642464E
:10988000494604F14400FFF7AFFA51463430FFF780
:10989000CBF97838BDE8F88F70C3000810B50349DC
:1098A00040F8781BFFF7E2F9783810BD70C3000864
:1098B0007047B838FFF7FEB87047000010B5F6F7EC
:1098C00041FD040004BF02A000F0A6FA204610BD2E
:1098D0004F70657261746F72206E6577206F75745A
:1098E000206F66206D656D6F72790D0A00000000B3
:1098F00003B401984100009850EAC12018BF042029
:109900004A0D18BF40F0010040F2FF72B2EB515F08
:1099100008BF40F00200012808BF052002B07047D0
:109920002DE9F0410A4D0E4607462C682868B0F133
:10993000006F08D12146AC064FF4CA722046F7F7F3
:109940003FF92046286004EB87000664BDE8F081FB
:1099500008ED00E02DE9F0411C4617460E00804658
:1099600007D0054602E02846B0473D442046641E25
:10997000F9D24046BDE8F0810020F7F7FEBD0000B7
:109980000A2209210148FFF71BB8000048520020B5
:1099900010B584B00023172216211948FFF7E0FA0A
:1099A000184A1949F7F746F80520009003221421B8
:1099B000CDE901120623072204211448FFF73AFFDC
:1099C000104A1349F7F736F81248002410210460B2
:1099D00044608460C46000F0B5FA0F48214604601A
:1099E00044608460C46000F0ADFA0C481221046049
:1099F00044608460C46004B0BDE8104000F0A2BAC6
:109A0000CC5B002000000008898F0008A05C0020CB
:109A10009D9800085C5D00206C5D00207C5D00204E
:109A200002486A4620F00700704700006F7100206E
:109A300030380A2801D2012070470020704700000A
:109A40000328BCBF002070470749002201EB8001BA
:109A500051F80C0C41F80C2C002804BF4FF0FF30DB
:109A60007047016849680847900900200328BCBF77
:109A700000207047064901EB800050F80C0C0028CC
:109A800004BF4FF0FF307047016889690847000044
:109A9000900900200328BCBF01207047064901EB54
:109AA000800050F80C0C002804BF4FF0FF307047C6
:109AB0000168C96808470000900900202DE9F043BB
:109AC0000E4683B081466149F7F7D4F8604C10B375
:109AD00060494846F7F7CEF840B35F494846F7F784
:109AE000C9F870B35D4C2068002804BF201D2060B9
:109AF000251DA84204D0562259495A4800F09CFC22
:109B00002168594F002400BF57F8240028B3641C73
:109B1000102CF9D323E0206820B9032202215348F6
:109B200000F074FE03B00020BDE8F083206820B987
:109B3000032202214D4800F069FE03B00120BDE878
:109B4000F083FFE7206820B903220221474800F094
:109B50005DFE03B00220BDE8F083102C11D33F4816
:109B6000002904BF011D01600068A84204D05622EC
:109B70003B493C4800F060FC03B04FF0FF30BDE8CB
:109B8000F0834FF0FF3047F824003448002904BF29
:109B9000011D01600068A84204D0562230493148B6
:109BA00000F04AFC99F800004FF000083A2810D065
:109BB00049466846FFF716FB6846FFF700FB98B377
:109BC0006846FFF701FB0028684609D0FFF7E9FA6D
:109BD00022E06A4626A14846F6F790FD00981BE071
:109BE000FFF7D3FA00B316F0020F18BF022522D0F8
:109BF00016F00C0F18BF45F4007516F0040F18BFCF
:109C000045F4806506466846FFF7EAFA0146306883
:109C10002A4683683046984700281FBF47F824002B
:109C2000E01C03B0BDE8F08347F8248003B04FF098
:109C3000FF30BDE8F08316F0040F18BF0125D7D11F
:109C400016F0080F14BF09250025D1E7C4B200089B
:109C5000E0010020CBB20008D3B200080C020020C3
:109C60000CC50008F8C400089009002090080020E6
:109C70003A2570000328BCBF00207047064A02EB5B
:109C8000800050F80C0C002804BF4FF0FF307047E4
:109C900002681369002218479009002070B5144625
:109CA0000E46032813DA1248006820B90322022165
:109CB000104800F0ABFD0025002C06D9715D0D4861
:109CC00000F036FF6D1CAC42F8D820460DE00A4982
:109CD00001EB800050F80C0C002804BF4FF0FF305F
:109CE00070BD01680B6831469847201A70BD0000AE
:109CF000E0010020900800209009002070B5EFF3EB
:109D00001080012121EA000080F0010572B60D4C9F
:109D10006068002808BF25706068B0F1FF3F04D17B
:109D2000322209A110A000F087FB606828B125B994
:109D3000362205A116A000F07FFB6068401C606021
:109D400070BD0000FC0100206D6265642D646576C5
:109D50002F636F6D6D6F6E2F6D6265645F637269E7
:109D6000746963616C2E6300696E746572727570DC
:109D7000745F656E61626C655F636F756E7465724A
:109D8000203C2055494E5433325F4D41580000006D
:109D9000696E74657272757074735F646973616201
:109DA0006C65640010B50E4C6068002808BF10BDDB
:109DB000EFF31080012121EA000090F0010F04D19F
:109DC000472208A10FA000F037FB6068401E6060CA
:109DD0006068002806BF2078002810BD62B610BD5C
:109DE000FC0100206D6265642D6465762F636F6DE4
:109DF0006D6F6E2F6D6265645F6372697469636114
:109E00006C2E6300696E74657272757074735F6432
:109E1000697361626C6564000FB410B503A90298A0
:109E200000F0B4FB012000F001F8000004460548F2
:109E3000F6F743FD0448F6F740FD002C18BF00F08C
:109E400025FBFEE7A0700020F4700020004870475A
:109E5000BCB2000870B50446B0F900000D46B0F180
:109E6000FF3F04D1462209A117A000F0E5FAB4F99A
:109E70000000012D04D0BDE87040002100F0B4BB0B
:109E8000BDE87040012100F0AFBB00006D62656469
:109E90002D6465762F746172676574732F68616CC9
:109EA0002F5441524745545F53544D2F544152470C
:109EB00045545F53544D333246342F6770696F5F9A
:109EC0006170692E630000006F626A2D3E70696EDA
:109ED00020213D202850696E4E616D65294E43005A
:109EE00070B50C4605460180B1F1FF3F08BF70BD5B
:109EF000C4F30310FAF7CAFC06460021204600F01E
:109F000073FB04F00F00012101FA00F0686006F114
:109F10001000A8600830E86070BD70B500260546E6
:109F20000C46FFF7DDFFB4F1FF3F08BF70BD002115
:109F30002846FFF78FFF31462846BDE8704000F005
:109F40009BB9000070B504460D460026FFF7C8FF18
:109F5000B5F1FF3F08BF70BDB4F90000B0F1FF3F9D
:109F600005D10A49342201F1400000F065FAA088C9
:109F7000E1680004086001212046FFF76BFF3146CD
:109F80002046BDE8704000F077B90000E09F00086F
:109F90002DE9F04104460E4600271546FFF7A0FFC5
:109FA000B6F1FF3F08BFBDE8F081B4F90000B0F1A1
:109FB000FF3F04D134220AA119A000F03DFA002D80
:109FC00012BF6068A0880004E16808600121204693
:109FD000FFF740FF39462046BDE8F04100F04CB99C
:109FE0006D6265642D6465762F7461726765747344
:109FF0002F68616C2F5441524745545F53544D2F85
:10A000005441524745545F53544D333246342F67C1
:10A0100070696F5F6F626A6563742E68000000008C
:10A020006F626A2D3E70696E20213D202850696E56
:10A030004E616D65294E43000121002000F020B9DA
:10A040000121084600F01CB90121022000F018B9D6
:10A050000121032000F014B90121042000F010B9FF
:10A060000521084600F00CB90621084600F008B9A1
:10A0700070B504464068104A00EB400101EB001047
:10A080000C49012301EB8000217B002501F00F0129
:10A0900052F8211002688B409A43026000EB810065
:10A0A00029464560C5614563B4F90C0000F09CFA8F
:10A0B000A56070BD5C040020A00100202DE9F84FD0
:10A0C0009A4693460F468046B1F1FF3F04BF4FF0DA
:10A0D000FF30BDE8F88FC7F3031007F00F09B9F19F
:10A0E000100F5DD2DFE809F0080C1014181C1C1CBE
:10A0F0001C1C20202020202006242D4E002516E0A8
:10A1000007242C4E012512E008242B4E02250EE0D8
:10A1100009242A4E03250AE00A24294E042506E0D4
:10A120001724284E052502E02824274E0625FAF795
:10A13000ADFB00900721384600F056FA3146204624
:10A14000FFF7EEFB04F01F00012202FA00F06109A4
:10A15000890001F1E021C1F8000188F800400020E9
:10A16000C8E9015005EB4500184900EB051001EB6B
:10A1700080001749A8F80C70036851F829108A402C
:10A180001A4300EB81010260C1F804A00098C1F8F5
:10A190003490C8610F48C0F800B00020BDE8F88FC7
:10A1A0000DA0FFF739FE4FF0FF30BDE8F88F00003B
:10A1B00039A0000841A0000849A0000851A00008EB
:10A1C00059A0000861A0000869A000085C040020F4
:10A1D000A00100209C010020496E746572727570A8
:10A1E00074496E206572726F723A2070696E206ECB
:10A1F0006F7420737570706F727465642E0A00003E
:10A2000030B40B460C21012402254FF0000CB2B1F2
:10A210000322012B02D0022B0BD01DE08168022902
:10A2200018BF032902D10821826015E0062184604D
:10A2300012E08168012918BF032914D1F3E7012B2B
:10A2400002D0022B12D007E08268022A18BF032A2C
:10A2500009D000BFC0F808C0B0F90C0030BC6CF3E6
:10A260001F1100F0C1B907218560F5E78268012A56
:10A2700018BF032AEED1D9E7B0F9000000F004BA04
:10A280002DE9F0470E0000EB400101EB00101949E9
:10A290004FF0000401EB800508BFBDE8F0870127FF
:10A2A000DFF85480DFF85490296807FA04F001427F
:10A2B0001AD005EB8400D8F8003090F83420C1693A
:10A2C00007FA02F213420FD0C8F80020406858B1D4
:10A2D0000969114204D1D9F800200221904703E016
:10A2E000D9F8002001219047641CB442DCD3BDE8BA
:10A2F000F08700005C040020143C01409C01002019
:10A3000010B5144C016821600A6822F040020A600E
:10A31000016961608169E1610021A160C2686261D7
:10A32000826822610722C4E90A124268E26021625F
:10A3300040696162A0612046F9F7E6FF00281CBF72
:10A3400005A0FFF769FD2068016841F04001016048
:10A3500010BD0000DC08002043616E6E6F74206940
:10A360006E697469616C697A652053504900000018
:10A3700010B5194A416802EB8114016821608168B7
:10A380006160C168A1600169E16041692161016AA0
:10A39000A1610021E161E184A184E185A185B0F999
:10A3A0001A10B1F1FF3F04BF0820606107D0B0F977
:10A3B0001800B0F1FF3F0CBF04200C206061FAF7D9
:10A3C000D5FA2046FAF784F9002808BF10BD03A08B
:10A3D000BDE81040FFF720BD9006002043616E6E7F
:10A3E0006F7420696E697469616C697A6520554182
:10A3F00052540A000D480178102905D1FF21FBF7BE
:10A40000F7FE0B4840688047FBF77CFF0948FDF7E3
:10A4100055FC0848FDF7D8FB0648FDF773FC0028FB
:10A420001CBF0448FDF71EFCF3E700000010010804
:10A430000000FF1F4852002070B514460D46064626
:10A44000FFF75CFC23462A46314603A000F074F86F
:10A45000BDE8704000F01AB86D62656420617373E6
:10A460006572746174696F6E206661696C65643AC7
:10A470002025732C2066696C653A2025732C206C8E
:10A48000696E65202564200A0000000084B0FFF793
:10A4900035FC05216846FFF755FD00BFBDF90000FA
:10A4A000B0F1FF3F04D134220DA11DA0FFF7C4FF7E
:10A4B000039901980860962000F068FDBDF900003E
:10A4C000B0F1FF3F04D1342205A115A0FFF7B4FF7E
:10A4D0000198039900040860962000F057FDDDE71D
:10A4E0006D6265642D6465762F746172676574733F
:10A4F0002F68616C2F5441524745545F53544D2F80
:10A500005441524745545F53544D333246342F67BC
:10A5100070696F5F6F626A6563742E680000000087
:10A520006F626A2D3E70696E20213D202850696E51
:10A530004E616D65294E43000FB470B5A0B025ACD7
:10A54000249DFFF7DBFB224629466846F5F764FFAA
:10A55000051E10DD0B48006820B9032202210A48BD
:10A5600000F054F900246E460748315D00F0E0FA2F
:10A57000641CAC42F8DBFFF715FC20B070BC5DF842
:10A5800014FB0000E00100209008002070B5A0B08E
:10A590000C460546FFF7B2FB224629466846F5F70A
:10A5A0003BFF051E10DD0A48006820B90322022186
:10A5B000084800F02BF900246E460648315D00F093
:10A5C000B7FA641CAC42F8DBFFF7ECFB20B070BDBF
:10A5D000E001002090080020704710B5FAF7C6F996
:10A5E000BDE81040F8F7B4BDF0B585B00C4605469F
:10A5F000B0F1FF3F04D181220FA11DA0FFF71CFF86
:10A6000004F00F07C4F30216C5F30310C4F3C31418
:10A6100005F00F05FAF73AF90121A940009119490F
:10A6200051F82710CDE901160321CDE9031469463D
:10A63000F8F778FC05B0F0BD6D6265642D64657651
:10A640002F746172676574732F68616C2F54415267
:10A650004745545F53544D2F5441524745545F531F
:10A66000544D333246342F70696E6D61702E630025
:10A6700070696E20213D202850696E4E616D6529FC
:10A680004E43000054B2000870B50C460546B0F1C8
:10A69000FF3F04D1A6220CA119A0FFF7CDFEC5F300
:10A6A000031005F00F05FAF7F1F8022C88BF00241B
:10A6B000C268690003238B409A43C260C26804FAEF
:10A6C00001F11143C16070BD6D6265642D646576F2
:10A6D0002F746172676574732F68616C2F544152D7
:10A6E0004745545F53544D2F5441524745545F538F
:10A6F000544D333246342F70696E6D61702E630095
:10A7000070696E20213D202850696E4E616D65296B
:10A710004E430000884208BF7047B0F1FF3F04BFBE
:10A720000846704710B5B1F1FF3F08BF10BD03A048
:10A73000FFF772FB4FF0FF3010BD000070696E6DC7
:10A740006170206D69732D6D617463680000000095
:10A7500010B5B0F1FF3F08BF10BDB1F90020B2F154
:10A76000FF3F0DD0B1F90020824204D14C68B4F112
:10A77000FF3F0AD106E031F90C2FB2F1FF3FF1D1D2
:10A780004FF0FF3402A0FFF747FB204610BD00004A
:10A7900070696E6D6170206E6F7420666F756E6487
:10A7A00020666F72207065726970686572616C00F6
:10A7B00010B50446B0F1FF3F08BF10BDB1F900006D
:10A7C000B0F1FF3F13D000BFB1F90000A04209D1A2
:10A7D00089682046FFF708FF2046BDE810400021A9
:10A7E000FFF752BF31F90C0FB0F1FF3FECD1BDE8DC
:10A7F000104001A0FFF710BB636F756C64206E6F93
:10A80000742070696E6F7574000000002DE9F843C4
:10A810000F46044616464B493846FFF799FF054652
:10A8200049493046FFF794FF01462846FFF772FF7B
:10A830002060B0F1FF3F04D16A2244A152A0FFF78B
:10A84000FBFD20684FF00108A0F18042B2F588427C
:10A850004FF000051AD053495348B2F54C4F03D07E
:10A86000B2F5504F27D038E00A6842F010020A6073
:10A870000A6822F010020A60016841F010010160CC
:10A88000006800F010000090656026E0474801680D
:10A8900041F400310160016821F400310160444855
:10A8A000016841F400310160006800F4003000905C
:10A8B000C4F8048011E00A6842F020020A600A68C5
:10A8C00022F020020A60016841F020010160006866
:10A8D000052100F02000009061601A493846FFF71A
:10A8E00067FF19493046FFF763FFB7F1FF3F03D019
:10A8F00001213846FFF7C8FEB6F1FF3F03D0012122
:10A900003046FFF7C1FE4FF41651C4E90215256128
:10A9100065612562278320466683FFF729FD20684D
:10A92000A0F18041B1F5884118BFBDE8F883214806
:10A9300021464C22C0F80080BDE8F8431E48F6F7D7
:10A940003FB90000A0B00008E8B000086D6265647F
:10A950002D6465762F746172676574732F68616CFE
:10A960002F5441524745545F53544D2F5441524741
:10A9700045545F53544D333246342F7365726961C9
:10A980006C5F6170692E63006F626A5F732D3E7544
:10A9900061727420213D2028554152544E616D65ED
:10A9A000294E4300243802404438024020380240F7
:10A9B00040380240E001002090080020034B59601D
:10A9C0004068034941F8202070470000E001002062
:10A9D000700600202DE9F04304464068DFF84C8102
:10A9E00083B008EB801900270097D9F80000A66B08
:10A9F0003D46016811F0400F1CBFC16811F0400FC7
:10AA000006D0E16911F0040F1CBF01F004010091B0
:10AA1000016811F0010F1CBF416911F0010F05D051
:10AA2000A18B009A01F4006111430091016811F0BB
:10AA3000020F1CBF416911F0010F05D0A18B009AD4
:10AA400001F4806111430091016811F0080F1CBFEF
:10AA5000406910F0010F05D0A08B009900F4007040
:10AA6000084300904846F9F7EBFC009810F4006F9B
:10AA700001BF009810F4806F009810F4007F51D14E
:10AA8000B9F82C0018B1B9F82E10411A2164B9F8A0
:10AA90002E0050B9D4E90F01401E814205D3A08B8E
:10AAA000009900F4807008430090A08B10F4005FC0
:10AAB00018BF002E36D0226C002A88BF94F84800B8
:10AAC00030D9715D814229D12564A08B009900F4B1
:10AAD000005008430090606808EB80100168CA6865
:10AAE00022F02002CA600168CA6822F48072CA603B
:10AAF00001684A6922F001024A6102686FF0200190
:10AB00001160016849680191C78590F83A102329BE
:10AB100014BF2021212180F83A1003E0691CCDB236
:10AB2000AA42CED8009803B0BDE8F083900600207A
:10AB30004268074800EB821318680268C2F3C0122B
:10AB4000002AFAD0C1F30800196848607047000075
:10AB50009006002030B44FF0000C102906BF4FF4CF
:10AB600000614160C0F804C0002A04BFC0F808C0FA
:10AB7000C0F80CC00CD00121012A08BFC0E902C1F5
:10AB800006D00224022A14BFC0E90241C0E9024CE7
:10AB90004169B1F5007F07D0002B08BF4FF4802C2E
:10ABA000C0F814C003D000E00BB1002101E04FF465
:10ABB0008271016130BCFFF7A3BB00002DE9F041B9
:10ABC000074600680024A0F560500E462546B0F107
:10ABD000804018BFB0F5806F0CD0B0F5784F18BF2B
:10ABE000B0F57C4F03D012A0FFF716F90BE0F9F790
:10ABF00073F901E0F9F758F9044604E004EBD47066
:10AC00004410681CC5B2B44201DD082DF6D3082DEE
:10AC100006D80D4800EB450030F8020CB86102E0A0
:10AC20000AA0FFF7F9F83846BDE8F041FFF768BB26
:10AC300053504920696E7374616E6365206E6F7442
:10AC4000207365740000000088B20008436F756CC3
:10AC5000646E2774207365747570207265717565F4
:10AC60007374656420535049206672657175656E12
:10AC7000637900002DE9F84F894604461F46904647
:10AC8000464948460A9EFFF763FD00904449404606
:10AC9000FFF75EFD824643493846FFF759FD83467C
:10ACA00041493046FFF754FD054651460098FFF7ED
:10ACB00031FD824629465846FFF72CFD0146504695
:10ACC000FFF728FD2060B0F1FF3F04D1512237A1EA
:10ACD00045A0FFF7B1FB216849480025A1F180425A
:10ACE000B2F5983207D1016841F4805101600168E2
:10ACF00001F48051009122684249A2F18043B3F5EA
:10AD0000605307D10A6842F480420A600A6802F47C
:10AD1000804200922268A2F18043B3F5705307D1BC
:10AD20000A6842F400420A60096801F40041009197
:10AD30002168A1F18042B2F59A3207D1016841F44D
:10AD400000510160006800F400500090134948462B
:10AD5000FFF72EFD12494046FFF72AFD11493846FC
:10AD6000FFF726FD6560A5603820E560A061A4F8C6
:10AD70001C80A4F81E9027846684B6F1FF3F04BFB0
:10AD80004FF40070606103D007493046FFF710FDB3
:10AD90002046BDE8F84FFFF7B3BA000030B1000815
:10ADA00078B10008C0B1000808B200086D6265649F
:10ADB0002D6465762F746172676574732F68616C9A
:10ADC0002F5441524745545F53544D2F54415247DD
:10ADD00045545F53544D333246342F7370695F616D
:10ADE00070692E63000000006F626A2D3E73706907
:10ADF00020213D20285350494E616D65294E430066
:10AE000044380240403802400A4AD0F800C0036883
:10AE100013609B68C3F34003002BF8D089B2CCF8D1
:10AE20000C10036801681160896811F0010FF9D0F6
:10AE3000D8687047DC08002010B504460068C06878
:10AE40008047606840680028206811D040688047CB
:10AE500061680246486803689A1A002A0CDC826816
:10AE60004A606168096800291CBF40688847E8E7B4
:10AE70008068BDE81040004748682168006809699B
:10AE8000BDE81040084700684068004770B5164CA0
:10AE90002068016911F0020F1CBFC16811F0020F98
:10AEA00004D06FF00201016100F048F820680169E8
:10AEB00011F0040F1ABFC16811F0040F70BD6FF0DC
:10AEC000040101612068456A084E3068281AB0F50F
:10AED0007A7F38BF70BDF8F733F9216805F57A70CD
:10AEE0008863356070BD00002004002094010020BC
:10AEF00002496FF002000968086170475409002098
:10AF000003480068C16821F00201C1607047000079
:10AF10005409002006480168002918BF7047012124
:10AF200001600549034808600020F8F72BB90000CC
:10AF3000EC010020000C0040540900200148FFF7FC
:10AF40007BBF0000BCB20008074810B5016839B9E2
:10AF5000012101600649054808600020F8F712F950
:10AF60000448006810BD0000EC010020000C004007
:10AF700054090020240C0040034909684863C8684C
:10AF800040F00200C86070475409002070B54FF4CB
:10AF90007A7100FB01F5FFF7D7FF0446FFF7D4FFF6
:10AFA000001BA842FAD370BD70B50546FFF7CCFF71
:10AFB0004FEA0004FFF7C8FF001BA842FAD370BD98
:10AFC00010B500290AD00878002807D00548784431
:10AFD000F5F750FE002801D0002010BD024878444B
:10AFE00010BD00007A1500007215000010B5002990
:10AFF0000AD00878002807D005487844F5F73AFECB
:10B00000002801D0002010BD0248784410BD000087
:10B010006A1500006215000010B50446006800289B
:10B0200006BF201D20602068211D884204D05622C2
:10B0300002490348FFF700FA206810BD0CC500085C
:10B04000F8C400084A68096800EB620012F0010FBA
:10B0500001D002685158084730B4002804BF30BC02
:10B06000704713684BB1526800EB620012F0010F99
:10B0700001D00268D35830BC1847D2F804C01CF085
:10B08000010F18BFBCF1000FEDD130BC70474FF07D
:10B090004070E1EE100A7047F6F7B5BBF6F7EABC70
:10B0A000020000000044004093030000090000007B
:10B0B00000100140930300000B0000000014014049
:10B0C000130400001600000000100140930300006C
:10B0D000260000000014014013040000FFFF0000E0
:10B0E000FFFFFFFF000000000300000000440040DD
:10B0F000930300000A0000000010014093030000C9
:10B100000C000000001401401304000017000000B0
:10B1100000100140930300002700000000140140CC
:10B1200013040000FFFF0000FFFFFFFF000000000E
:10B1300007000000003001409302000015000000ED
:10B1400000300140930200001F0000000038004062
:10B15000930200002300000000380040930200002A
:10B160002C000000003C004013030000FFFF000023
:10B17000FFFFFFFF0000000006000000003001405C
:10B180009302000014000000003001409302000010
:10B190001E00000000380040930200002200000062
:10B1A00000380040930200002B000000003C0040EB
:10B1B00013030000FFFF0000FFFFFFFF000000007F
:10B1C0000500000000300140930200001300000061
:10B1D00000300140930200001A00000000380040D7
:10B1E000930200001D0000000038004093020000A0
:10B1F0002A000000003C004013030000FFFF000095
:10B20000FFFFFFFF000000000400000000300140CD
:10B21000830200000F0000000030014083020000A4
:10B220001900000000380040830200001C000000EC
:10B230000038004083020000FFFF0000FFFFFFFF17
:10B2400000000000000000000000000001020304F4
:10B2500006070809000000000100000011000000BE
:10B2600002000000120000000300000000001110A6
:10B270000000211000003110000012100000221008
:10B28000000032100000001000000800100018003C
:10B2900020002800300038000000000001020304F4
:10B2A000010203040607080915AF000849AF0008AA
:10B2B00001AF0008F1AE000879AF0008A8B200089D
:10B2C000040200202F737464696E002F7374646F1E
:10B2D0007574002F7374646572720000D98A000857
:10B2E000000000000000000000000000111111111A
:10B2F00011111111102056657273696F6E3A20306A
:10B300002E310000FF0000000200000000000000DD
:10B31000FF0007000100000000000000FF01000026
:10B320000801000067000000FF020000100000009C
:10B3300000000000FF040000080000000000000002
:10B34000FF0500000800000000000000FF060000EC
:10B350000800000000000000FF07000008000000D7
:10B3600000000000FF0800000801000000000000CD
:10B37000FF0900000800000000000000FF0A0000B4
:10B380000800000000000000FF0B000008000000A3
:10B3900000000000FF0C0000100100000000000091
:10B3A000FF0E00000801000000000000FF0F000079
:10B3B0000801000000000000FF1000000100000074
:10B3C00000000000FF10010001000000000000006C
:10B3D000FF1002000100000000000000FF10030049
:10B3E0000100000000000000FF110000010000004B
:10B3F00001000000FF110100010000000100000039
:10B40000FF1200000100000000000000FF12010018
:10B410000100000000000000FF1202000100000017
:10B4200000000000FF120300010000000000000007
:10B43000FF1300000101000000000000FF130100E5
:10B440000101000000000000FF14000001010000E5
:10B4500000000000FF1401000101000000000000D6
:10B46000FF1402000101000000000000FF140300AF
:10B470000101000000000000FF14040001010000B1
:10B4800000000000FF1500000101000000000000A6
:10B49000FF1501000101000000000000FF1502007F
:10B4A0000101000000000000FF1503000101000081
:10B4B00000000000FF150400010100000000000072
:10B4C000FF1505000101000000000000FF15060047
:10B4D0000101000000000000FF150700010100004D
:10B4E00000000000FF160000010100000000000045
:10B4F000FF1601000101000000000000FF1602001D
:10B500000101000000000000FF160300010100001F
:10B5100000000000FF160400010100000000000010
:10B52000FF1605000101000000000000FF160600E4
:10B530000101000000000000FF16070001010000EB
:10B5400000000000FF1700000101000000000000E3
:10B55000FF1701000101000000000000FF170200BA
:10B560000101000000000000FF17030001010000BE
:10B5700000000000FF1704000101000000000000AF
:10B58000FF1705000101000000000000FF17060082
:10B590000101000000000000FF170700010100008A
:10B5A00000000000FF180000010100000000000082
:10B5B000FF1801000101000000000000FF18020058
:10B5C0000101000000000000FF180300010100005D
:10B5D00000000000FF18040001010000000000004E
:10B5E000FF1805000101000000000000FF18060020
:10B5F0000101000000000000FF1807000101000029
:10B6000000000000FF190000010100000000000020
:10B61000FF1901000101000000000000FF190200F5
:10B620000101000000000000FF1A000001010000FD
:10B6300000000000FF1A01000101000000000000EE
:10B64000FF1A02000101000000000000FF1A0300C1
:10B650000101000000000000FF1A040001010000C9
:10B6600000000000FF1A05000101000000000000BA
:10B67000FF1A06000101000000000000FF1A070089
:10B680000101000000000000FF1B0000040000009A
:10B6900000000000FF1C000004000000000000008B
:10B6A000FF1D00000500000000000000FF1E00005C
:10B6B0000501000000000000FF1F00000500000061
:10B6C00000000000FF200000080100000000000052
:10B6D000FF7D00000801000000000000FF7E000068
:10B6E0000801000001000000FF7F000001000000D1
:10B6F0000100000000210000010000000000000027
:10B7000000210100010000000100000000210200F2
:10B710000100000000000000002103000100000003
:10B7200000000000002104000100000000000000F3
:10B7300000210500010000000000000000220000C0
:10B7400004000000070000000023000008000000C3
:10B75000F0000000002400010D00000080FEFFFF4B
:10B76000002600010D00000080FFFFFF00280001FF
:10B770000D00000080000000002A00010D00000004
:10B7800080010000002C00010D00000080FEFFFF82
:10B79000002E00010D00000080FFFFFF00300001BF
:10B7A0000D00000080000000003200010D000000CC
:10B7B00080010000003400010D00000000000000C6
:10B7C000003600010D0000000000000000400000F5
:10B7D0000100000000000000004001000400000023
:10B7E000070000000041000007000000000000000A
:10B7F00000420000070000000000000000430000BD
:10B8000007000000000000000044000007000000E6
:10B8100000000000004500000700000000000000DC
:10B820000046000007000000000000000047000084
:10B8300007000000000000000048000007000000B2
:10B8400000000000004900000100000000000000AE
:10B850000049010001000000010000000049020051
:10B860000100000001000000004903000100000089
:10B870000100000000490400010000000100000078
:10B880000049050001000000010000000049060019
:10B890000100000001000000004A00000400000058
:10B8A00004000000004A040004000000040000003E
:10B8B000004B00000400000004000000004B0400E6
:10B8C0000400000004000000004C00000400000020
:10B8D00004000000004C040004000000040000000C
:10B8E000004D00000400000004000000004E0000B5
:10B8F0000400000004000000004E040003000000EB
:10B9000005000000005100000C00000000000000D5
:10B91000005300000C000000FC0F00000055000068
:10B9200008000000070000000056000008000000AA
:10B9300000000000005700000801000000000000A7
:10B94000005800000801000000000000005900003D
:10B95000010000000100000000590100010000008A
:10B9600001000000005A000001000000000000007B
:10B97000005A01000300000000000000005B00000E
:10B980000800000000000000005C0000080000004B
:10B990001D000000005D000006000000090000001E
:10B9A000005E00000200000002000000005E0200D5
:10B9B0000200000001000000005E04000200000020
:10B9C00000000000005F0000040000000100000013
:10B9D000005F04000400000002000000006000009E
:10B9E000100000000A0000000062000001000000DA
:10B9F00001000000006201000100000001000000E1
:10BA00000063000004000000080000000063040060
:10BA100002000000020000000064000007000000B7
:10BA2000000000000065000008000000FF000000AA
:10BA30000066000001000000010000000067000037
:10BA40000800000000000000006800000400000082
:10BA50000800000000680400040000000700000067
:10BA600000690100010000000100000000690200FF
:10BA70000100000001000000006903000100000057
:10BA800001000000006A0000010000000100000049
:10BA9000006A01000100000001000000006A0200CD
:10BAA0000100000000000000006A03000100000027
:10BAB00000000000006A0400010100000000000016
:10BAC000006A05000101000000000000006A060095
:10BAD0000100000000000000006A070001000000F3
:10BAE00000000000006B00000800000001000000E2
:10BAF000006C00000800000020000000006D000045
:10BB00000800000064000000006E00000800000053
:10BB100064000000006F0000050000000700000046
:10BB2000007000000500000005000000007100002A
:10BB30000500000008000000007200000600000080
:10BB4000000000000073000006000000000000007C
:10BB500000740000060000000000000000740600F1
:10BB60000100000000000000007500000600000059
:10BB700000000000012100000100000000000000A2
:10BB8000012101000100000000000000012102006D
:10BB90000100000000000000012200001000000071
:10BBA000000000000124000004000000010000006B
:10BBB0000124040004000000020000000125000030
:10BBC0000300000000000000012700010800000041
:10BBD0000000000001280001080000000000000033
:10BBE00001290000010000000000000001290100FF
:10BBF0000400000000000000012905000100000011
:10BC00000000000001290600010000000000000003
:10BC1000012A00000200000000000000012A0200CA
:10BC20000300000005000000012A050002000000DA
:10BC300000000000012A07000100000001000000D0
:10BC4000012B00000100000000000000012B01009A
:10BC50000100000000000000012B020003000000B2
:10BC600000000000012C000008000000000000009F
:10BC7000012D00000100000001000000012E000065
:10BC80000400000001000000012E04000400000078
:10BC900002000000012F0000100000000A00000058
:10BCA000013100000100000001000000013101002D
:10BCB0000100000001000000013200000800000047
:10BCC0000A00000001330000030000000300000030
:10BCD00001340000080000001D00000001350000D4
:10BCE0000600000024000000013600000C000000E7
:10BCF0000000000001380000020000000200000007
:10BD000001380200020000000100000001380400B8
:10BD100002000000000000000139000008000000DF
:10BD200000000000013A00000200000000000000D6
:10BD3000013A02000100000000000000013A030087
:10BD40000100000001000000013B000004000000B1
:10BD500008000000013B0400020000000300000096
:10BD6000013B06000100000000000000013C000053
:10BD70000400000007000000013C04000100000076
:10BD800001000000013D000008000000FF0000006D
:10BD9000013E00000801000080000000013F00009B
:10BDA0000300000000000000013F0300030000004A
:10BDB00000000000013F060001000000000000003C
:10BDC000013F0700010000000000000001400000EA
:10BDD000030000000000000001400300010000001B
:10BDE000000000000140040002000000000000000C
:10BDF00001400600010000000000000001410000B9
:10BE000005000000000000000141070001000000E3
:10BE100000000000014200001000000000000000CF
:10BE20000144000020000000000000000148000064
:10BE30002000000000000000014C0000080000008D
:10BE400000000000014D00000100000001000000A2
:10BE5000014D01000200000000000000014D030040
:10BE60000100000001000000014D0400010000007D
:10BE700000000000014D050003000000000000006C
:10BE80000150000008000000000000000151000007
:10BE90000800000000000000015200000100000046
:10BEA00001000000015300000A0000000000000033
:10BEB0000221000008000000000000000222000033
:10BEC000080100000000000002230000080000003C
:10BED000000000000225000001000000000000003A
:10BEE00002260000080000000000000002270000F9
:10BEF0000801000000000000022800000800000007
:10BF000000000000022A0000010000000000000004
:10BF1000022B00000100000000000000022B0100C5
:10BF20000100000000000000022B020001000000E0
:10BF300001000000022B03000100000000000000CF
:10BF4000022B04000100000000000000022B05008D
:10BF50000100000000000000022B060001000000AC
:10BF600000000000022C00000200000000000000A1
:10BF7000022D00000400000002000000022D040059
:10BF80000400000004000000022E00000400000075
:10BF900002000000022E0400040000000400000063
:10BFA000022F00000500000000000000022F050025
:10BFB0000100000000000000022F06000100000048
:10BFC00000000000022F0700010000000000000038
:10BFD00002300000100000000000000002330000EA
:10BFE0000801000000000000023400000801000009
:10BFF0000000000002360000080100000000000000
:10C0000002380000080100000000000002390000B2
:10C010000801000000000000023A000008010000D2
:10C0200000000000023B00000801000000000000CA
:10C03000023C00000801000000000000023D00007A
:10C040000801000000000000023E0000080100009E
:10C0500000000000023F0000080100000000000096
:10C060000240000008010000000000000241000042
:10C070000801000000000000024200001001000062
:10C080000000000002440000100100000000000059
:10C09000024600002001000000000000024A0000EB
:10C0A0000401000000000000024A04000401000036
:10C0B00000000000024B000004010000000000002E
:10C0C000024B04000401000000000000024C0000CC
:10C0D0000401000000000000024C04000401000004
:10C0E00000000000024D00000401000000000000FC
:10C0F000024D04000401000000000000024E000098
:10C100000401000000000000024F000003010000D5
:10C1100000000000024F03000301000000000000C7
:10C120000250000008000000000000000251000062
:10C1300008000000000000000252000001000000A2
:10C140000000000002520100010000000000000099
:10C150000252020001000000000000000253000033
:10C160000100000000000000025400000100000077
:10C170000000000002540100010000000000000067
:10C1800002540200020000000000000002540400FB
:10C19000030000000000000002540700010100003D
:10C1A0000000000002550000080000000000000030
:10C1B00002560000080000000000000002570000C6
:10C1C0000801000000000000025800000801000003
:10C1D0000000000002590000010000000000000003
:10C1E000025901000100000001000000025A000194
:10C1F0000800000000000000025B020106000000D1
:10C2000000000000025C00011000000000000000BF
:10C21000025E00000401000000000000025F000058
:10C2200005010000000000000260000005010000A0
:10C230000000000002610000050100000000000095
:10C240000121000008000000000000008D96000899
:10C25000000000003031323334353637383941424E
:10C260004344454640305800303132333435363758
:10C270003839616263646566403078000400000804
:10C28000000000000000000200010000100000009B
:10C290000000000000000000303132333435363702
:10C2A00038396162636465667870003031323334E6
:10C2B000353637383941424344454658500000002E
:10C2C00002400000000000A0000000000540000047
:10C2D000000000C8000000000C4000000000409C6E
:10C2E00000000000194000000020BCBE000000005B
:10C2F00034400000BFC91B8E00000004B5400000A0
:10C30000504BCFD06607E2CF010000006C41000027
:10C310003E8251AADFEEA73401000000D94200009E
:10C32000DCB5A0E23A301F97FFFFFFFFB4450000E5
:10C33000FD25A0C8E9A3C14FFFFFFFFFFF3F00009D
:10C340000000008000000000FF3F000000000080AF
:10C35000000000000000000000000000259200081E
:10C3600051920008599200080000000000000000EF
:10C3700061950008000000000000000079990008A5
:10C380007999000879990008799900087999000845
:10C3900079990008E9890008418A00080000000036
:10C3A0003B8A00083D8A00080000000000000000F1
:10C3B000000000000000000000000000000000007D
:10C3C00000000000000000006D8C0008000000006C
:10C3D0000000000000000000B98C00088D8C0008EF
:10C3E000698D00080000000000000000000000004F
:10C3F000000000000000000000000000898F00081D
:10C4000000000000000000000000000048FFFFFFE7
:10C4100000000000BD8F0008B58F0008000000007C
:10C42000F98F0008B98F000800000000B18F0008E4
:10C430000000000000000000B1980008B998000852
:10C44000B39800080000000044FFFFFF0000000058
:10C4500000000000000000000000000000000000DC
:10C46000BD8F0008B58F000800000000F98F00089C
:10C47000B98F000800000000B18F00083D9000084F
:10C48000000000003B8A00083D8A000879990008F6
:10C4900079990008FCFFFFFF000000000000000089
:10C4A0000000000000000000000000000D910008E6
:10C4B0000000000000000000000000007999000862
:10C4C0007999000879990008799900087999000804
:10C4D00079990008E98900087991000800000000B6
:10C4E0003B8A00083D8A0008FCFFFFFF00000000B7
:10C4F00000000000000000005F707472203D3D20CD
:10C500002854202A29265F64617461006D62656485
:10C510002D6465762F6170692F53696E676C657441
:10C520006F6E5074722E68007CC600089401002063
:10C530008C020000D001000868C700082004002019
:10C54000486D00002C0200081C00000043000000A1
:10C55000F8FFFFFF0C0000000E0000000F000000BD
:10C560002E0000001001000043000000F8FFFFFF54
:10C5700000404040404040404040414141414140F6
:10C5800040404040404040404040404040404040AB
:10C59000400502020202020202020202020202023A
:10C5A000022020202020202020202002020202023F
:10C5B0000202909090909090101010101010101097
:10C5C00010101010101010101010101002020202A3
:10C5D00002028888888888880808080808080808E7
:10C5E00008080808080808080808080802020202E3
:10C5F00040000000000000000000000000000000FB
:10C60000000000000000000000000000000000002A
:10C61000000000000000000000000000000000001A
:10C62000000000000000000000000000000000000A
:10C6300000000000000000000000000000000000FA
:10C6400000000000000000000000000000000000EA
:10C6500000000000000000000000000000000000DA
:10C6600000000000000000000000000000000000CA
:10C67000000000000DD3FFFF19D3FFFF51041CBDC4
:10C6800001053201320232030A150414091B41016B
:10C690002B3B0A06572A4060140902431302011C6F
:10C6A000C03209621B01020B130524161001052478
:10C6B000011009010424020205240617010705825E
:10C6C0000308151009040133020A1D07050102437E
:10C6D0002C070581070938442A40072A8107112BB6
:10C6E0000907440A2204440A16FF4413E3661408A7
:10C6F000FB681B0851044113C96D1B08E50C4B571F
:10C700006910811AFD181AF10413996E1408097042
:10C710001408E1621B08DD3C1A352C5A393C7201C1
:10C720001A09241A350413E16F1B0865081A41041D
:10C730001A15041AA5041E04030904128B1302021D
:10C740001E4083044057C15B020339690881041EFF
:10C75000C194C11502030A0E054603030E1B3202E3
:08C760001AFF010110000000A6
:040000050800019559
:00000001FF
